:10007C000E94173308950E9455330895249710E079
:10008C001093FF040FEF1FEF2FEF3FEF0093AC0423
:10009C001093AD042093AE043093AF04CF93DF9351
:1000AC0000E010E020E030E03A932A931A930A9390
:1000BC00EBEDF1E08F011A930A930E943E00DF9161
:1000CC00CF91EBEDF1E011911B3E10E009F01FEF29
:1000DC001F93EBEDF1E032961191103910E009F01D
:1000EC001FEF0F91102B112311F40C94D400E9E99C
:1000FC00F3E034961191143011F0163001F010E049
:10010C0009F41FEF1095112311F40C94930012E0D5
:10011C001093DA0110E00C944302E9E9F3E038960D
:10012C0011911093FF040FEF1FEF2FEF3FEF009390
:10013C00AC041093AD042093AE043093AF04CF9372
:10014C00DF9300E010E020E030E03A932A931A931A
:10015C000A93EBEDF1E08F011A930A930E943E0093
:10016C00DF91CF91EBEDF1E011911B3E10E009F026
:10017C001FEF1F93EBEDF1E032961191103910E067
:10018C0009F01FEF0F91102B112311F40C94D400D4
:10019C0011E01093DA0110E00C944302EBEDF1E066
:1001AC00FA93EA93E881F9813B96019111910093BE
:1001BC000B0510930C0500910B0510910C05D80143
:1001CC0020E230E0E89445F80E94873700930D0553
:1001DC0010930E05E881F9813E96019111910093DF
:1001EC00000510930105E881F98170961191109327
:1001FC000205E881F981769601911191009303052E
:10020C001093040500910005109101050F931F93A5
:10021C0010910205012F11270F931F9300910305D5
:10022C0010910405E89445F8BF91AF910E94653791
:10023C003F912F91020F131F009305051093060594
:10024C00E881F98171960191119100930705109342
:10025C00080500910705109108050F931F93009155
:10026C000D0510910E05E89445F8BF91AF910E94D1
:10027C00863700931605109317050091050510910C
:10028C0006050F931F930091070510910805A0E236
:10029C00B0E0E89445F80E9465370F931F930091E6
:1002AC000B0510910C05E89445F8BF91AF910E9495
:1002BC0086373F912F91020F131F0093090510935E
:1002CC000A05E881F981739601911191103009F4B6
:1002DC00003010E011F008F01FEF112311F40C9412
:1002EC008801E881F98173960191119133272227B6
:1002FC0000930F05109310052093110530931205F0
:10030C000C949701E881F981B0960191119121919A
:10031C00319100930F051093100520931105309324
:10032C00120500910F0510911005209111053091C7
:10033C00120540E052E060E070E0E89445F80E945D
:10034C00C1370093F7041093F8042093F904309309
:10035C00FA04E881F9813D961191109313050091EF
:10036C000F051091100520911105309112050F9376
:10037C001F932F933F930091090510910A05332782
:10038C002227015010402040304020953095109588
:10039C000095FF91EF91BF91AF910A0F1B1F2E1F7C
:1003AC003F1F0F931F932F933F9310911305012F12
:1003BC00112733272227E89445F80E9403380E5F53
:1003CC001F4F2F4F3F4F0093140510931505229686
:1003DC0000910B0510910C05169507950093BB0425
:1003EC001093BC04E4E2F4E0EF93FF9310E0E4E03C
:1003FC00F0E0BF91AF913196319711F01D93FCCF86
:10040C00E8E2F4E0EF93FF9310E0E4E8F0E0BF9152
:10041C00AF913196319711F01D93FCCF00910505EA
:10042C0010910605332722270093BD041093BE04B8
:10043C002093BF043093C004E1ECF4E0EF93FF93FE
:10044C003196FA93EA9315E11A9317EF41221FEBB9
:10045C0041221CE50E94F73615E11F9318810F917C
:10046C00011B102FFF91EF911083239610E0109336
:10047C00DA0111E010931F051FEF0895CF93DF935E
:10048C0000910005109101050F931F930091180521
:10049C00109119053F912F91020F131F332722271B
:1004AC003A932A931A930A93EBEDF1E08F011A9386
:1004BC000A930E943E00DF91CF910895CF93DF9372
:1004CC0000910005109101050F931F9300911805E1
:1004DC00109119053F912F91020F131F33272227DB
:1004EC003A932A931A930A93EBEDF1E08F011A9346
:1004FC000A930E944100DF91CF910895CF93DF932F
:10050C0000910005109101050F931F9300911805A0
:10051C00109119053F912F91020F131F0F931F93E9
:10052C0000910305109104053F912F91020F131FA9
:10053C00332722273A932A931A930A93EBEDF1E08F
:10054C008F011A930A930E944100DF91CF91089575
:10055C00088119810F931F930091BB041091BC0467
:10056C00E89445F8BF91AF910E9486370093180527
:10057C0010931905088119810F931F930091BB04E7
:10058C001091BC04E89445F8BF91AF910E94863756
:10059C008F01507821F0019509F41A95109500936C
:1005AC001A0510931B050E944402EBEDF1E0EF934A
:1005BC00FF9300911A0510911B05000F111FFF915D
:1005CC00EF91E00FF11F0191119108950A811B81A8
:1005DC000F931F930091BB041091BC04E89445F851
:1005EC00BF91AF910E94863700931805109319059F
:1005FC000A811B810F931F930091BB041091BC04C3
:10060C00E89445F8BF91AF910E9486378F015078DE
:10061C0021F0019509F41A95109500931A05109381
:10062C001B050E944402EBEDF1E0EF93FF93009168
:10063C001A0510911B05000F111FFF91EF91E00F90
:10064C00F11FEF93FF9308811981FF91EF910193B3
:10065C0011930E94640210910205123010E009F40B
:10066C001FEF112311F40C943D030E948402089592
:10067C000E94440200911805109119050F931F93C5
:10068C00009103051091040598011F910F91131708
:10069C0009F402171FEF08F01127112311F40C9421
:1006AC00E80300911A0510911B050F931F930091FD
:1006BC00BB041091BC0498011F910F91131709F4FE
:1006CC0002171FEF08F01127112311F40C94BA0331
:1006DC00EBEDF1E0EF93FF9300911A0510911B05E0
:1006EC00000F111FFF91EF91E00FF11F019111917C
:1006FC00103009F4003010E009F41FEF112311F44D
:10070C000C94AF03A0911A05B0911B051196A09300
:10071C001A05B0931B0500911805109119050F933C
:10072C001F930091BB041091BC04E89445F8BF9151
:10073C00AF910E9465370F931F9300911A0510918A
:10074C001B053F912F91020F131F015010400C9469
:10075C00EA03A0911A05B0911B051196A0931A05F6
:10076C00B0931B050C945703A0911805B091190573
:10077C001196A0931805B0931905009118051091C6
:10078C0019050F931F93009103051091040598010F
:10079C001F910F91131709F402171FEF08F011277F
:1007AC00112311F40C94E40310E000E000931A05FB
:1007BC0010931B050E9444020C94E6030C94E8036E
:1007CC000C9440031FEF0FEF089510E000E000932E
:1007DC0018051093190510E000E000931A0510930A
:1007EC001B050E943E0308953B812A8119810881D3
:1007FC000F931F932F933F930091090510910A05B6
:10080C0033272227D801F9013F912F911F910F9186
:10081C003F1729F42E1719F41B1709F40A1710E0C7
:10082C0008F01FEF1F9300910F05109110052091F8
:10083C001105309112050F931F932F933F933B811A
:10084C002A8119810881D801F9013F912F911F91BB
:10085C000F913F1729F42E1719F41B1709F40A17D7
:10086C0010E008F01FEF0F911023112311F40C94DA
:10087C0073043B812A81198108810F931F932F9355
:10088C003F930091090510910A0533272227015047
:10089C001040204030402095309510950095FF91E8
:1008AC00EF91BF91AF910A0F1B1F2E1F3F1F0F938C
:1008BC001F932F933F9310911305012F112733276B
:1008CC002227E89445F80E9403380E5F1F4F2F4FE4
:1008DC003F4F0C9477040C94770410E000E00C94D8
:1008EC0077040895088119810F931F9300911405C3
:1008FC001091150598011F910F91131709F4021708
:10090C001FEF10F009F011271F9308811981103087
:10091C0009F4013010E011F008F01FEF0F911023D3
:10092C00112311F40C94C404088119810250104055
:10093C00332722270F931F932F933F931091130567
:10094C00012F112733272227E89445F80E94B63748
:10095C000F931F932F933F930091090510910A0554
:10096C0033272227FF91EF91BF91AF910A0F1B1FE5
:10097C002E1F3F1F0C94CA040C94CA040FEF1FEFD8
:10098C002FEF3FEF0C94CA040895229710E01883C0
:10099C00FE013196FA93EA9311E0108318E01A9352
:1009AC001081088101171FEF08F01127112311F096
:1009BC000C942605FE013796EF93FF931C81012FB3
:1009CC00112701501040FF91EF91E00FF11F119191
:1009DC00103210E009F41FEF112311F40C94FA04F7
:1009EC000C9426050C941D05FE013396108113956D
:1009FC001083ED81FE81EF93FF931B81FF91EF91AB
:100A0C00012F1127E00FF11FEF93FF93FE01379693
:100A1C00EF93FF931C81012F112701501040FF9180
:100A2C00EF91E00FF11F1191FF91EF911193E9817B
:100A3C00FA81108113951083112311F00C94D704B3
:100A4C002396FE01349638961191103210E009F07D
:100A5C001FEF112311F40C949D05FE0110811395C9
:100A6C001083EA81FB81EF93FF931881FF91EF9143
:100A7C00012F1127E00FF11F1EE21193FE01319699
:100A8C00FA93EA9319E010831BE01A931081088102
:100A9C0001171FEF08F01127112311F00C949C057E
:100AAC00FE013796EF93FF931C81012F1127015004
:100ABC001040FF91EF91E00FF11F1191103210E0F7
:100ACC0009F41FEF112311F40C9470050C949C0580
:100ADC000C949305FE013396108113951083ED81D0
:100AEC00FE81EF93FF931B81FF91EF91012F112753
:100AFC00E00FF11FEF93FF93FE013796EF93FF93F7
:100B0C001C81012F112701501040FF91EF91E00F34
:100B1C00F11F1191FF91EF911193E981FA811081ED
:100B2C0013951083112311F00C944D052396EA8133
:100B3C00FB81EF93FF931881FF91EF91119308952F
:100B4C00239711E0198311E01A83FE013596EF9378
:100B5C00FF931981FF91EF91012F1127E00FF11FE6
:100B6C0011911E3210E009F41FEF112311F40C94B3
:100B7C00E0051A8119301FEF08F01127112311F429
:100B8C000C94DE05EB81FC81EF93FF931A81012F0E
:100B9C00112701501040FF91EF91E00FF11F10E26F
:100BAC001193FE0132961081139510830C94BF059E
:100BBC000C94D806FE013596EF93FF931981FF91A3
:100BCC00EF91012F1127E00FF11F11911A3210E054
:100BDC0009F41FEF112311F40C944B061A8910958C
:100BEC00112311F40C94FD0510E00C9418071A81D4
:100BFC0019301FEF08F01127112311F40C9427065C
:100C0C001A8119301FEF08F01127112311F40C94DD
:100C1C002506EB81FC81EF93FF931A81012F11279D
:100C2C0001501040FF91EF91E00FF11F1FE3119362
:100C3C00FE0132961081139510830C9406060C94C9
:100C4C0049061A811C301FEF08F01127112311F4EB
:100C5C000C944606EB81FC81EF93FF931A81012FD4
:100C6C00112701501040FF91EF91E00FF11F1FE38E
:100C7C001193FE0132961081139510830C94270664
:100C8C001FEF0C9418070C94D806FE013596EF93C1
:100C9C00FF931981FF91EF91012F1127E00FF11FA5
:100CAC0011911F3310E009F41FEF112311F40C9470
:100CBC007E061A891095112311F40C94680610E025
:100CCC000C941807EB81FC81EF93FF931A81012F91
:100CDC00112701501040FF91EF91E00FF11F1FE31E
:100CEC001193FE0132961081139510830C94D80643
:100CFC00FE013596EF93FF931981FF91EF91012F30
:100D0C001127E00FF11F11911C32D1F020F410309B
:100D1C0010F0442715C041E01E3291F01F3281F0D3
:100D2C00103471F020F41A3310F0442709C041E05C
:100D3C001F3F31F020F41F3710F0442701C041E071
:100D4C0010E009F41FEF112311F40C94B00610E01D
:100D5C000C941807EB81FC81EF93FF931A81012F00
:100D6C00112701501040FF91EF91E00FF11FEF930D
:100D7C00FF93FE013596EF93FF931981FF91EF914D
:100D8C00012F1127E00FF11F1191113618F01B37AD
:100D9C0008F41052FF91EF911193FE0132961081DD
:100DAC0013951083FE0131961081139510831981D0
:100DBC001F93FE01359610810F91011710E011F071
:100DCC0008F01FEF112311F40C94EE060C94F806A6
:100DDC001A811B3010E011F008F01FEF112311F4F1
:100DEC000C94AB051A811C301FEF08F0112711234E
:100DFC0011F40C941707EB81FC81EF93FF931A818C
:100E0C00012F112701501040FF91EF91E00FF11FBE
:100E1C0010E21193FE0132961081139510830C94FD
:100E2C00F8061FEF08952197FE01FA93EA9311E05B
:100E3C0010831BE01A931081088101171FEF08F033
:100E4C001127112311F00C947E07EE81FF81EF9393
:100E5C00FF931B81012F112701501040FF91EF913F
:100E6C00E00FF11F1191113618F01B3708F41052D6
:100E7C001F93EC81FD81EF93FF931B81012F1127B1
:100E8C0001501040FF91EF91E00FF11F11911136BD
:100E9C0018F01B3708F410520F91011710E009F0ED
:100EAC001FEF112311F40C947507EE81FF81EF9362
:100EBC00FF931B81012F112701501040FF91EF91DF
:100ECC00E00FF11F11911F3310E009F01FEF1123F8
:100EDC0011F40C94750710E023960C948007E981AB
:100EEC00FA81108113951083112311F00C942207B1
:100EFC0023961FEF089511E010931F053B812A8163
:100F0C001981088100932005109321052093220557
:100F1C003093230500912005109121052091220585
:100F2C00309123050F931F932F933F930091050549
:100F3C001091060533272227D801F9013F912F91F3
:100F4C001F910F913F1729F42E1719F41B1709F451
:100F5C000A1710E009F41FEF10931E0510911E05DF
:100F6C001095112311F40C94D707CF93DF930091B4
:100F7C0020051091210520912205309123053A93EB
:100F8C002A931A930A930E94FA03DF91CF9100934C
:100F9C0024051093250510E000E00093260510931E
:100FAC00270510E000E000931C0510931D05089523
:100FBC0010911F05139510931F0510911F051F937A
:100FCC0000910D0510910E05102F0F91011710E0D7
:100FDC0011F008F01FEF112311F40C94F40811E038
:100FEC0010931F05A0911C05B0911D051196A0939F
:100FFC001C05B0931D0510911E05112311F40C94C2
:10100C00380800911C0510911D050F931F9300913A
:10101C0016051091170598011F910F91131709F4DC
:10102C00021710E009F41FEF112311F40C9423089C
:10103C0010E00C94F5080C943608A0912005B091A2
:10104C002105E0912205F0912305119608F43196C3
:10105C00A0932005B0932105E0932205F09323057E
:10106C000C94F408A0912005B0912105E091220583
:10107C00F0912305119608F43196A0932005B093B6
:10108C002105E0932205F093230500912005109192
:10109C00210520912205309123050F931F932F9347
:1010AC003F930091090510910A053327222701501F
:1010BC001040204030402095309510950095FF91C0
:1010CC00EF91BF91AF910A0F1B1F2E1F3F1F0F9364
:1010DC001F932F933F9310911305012F1127332743
:1010EC002227E89445F80E9403388C01900150782F
:1010FC0041F0015010402040304020953095109523
:10110C000095303029F4203019F4103009F40030F7
:10111C0010E009F41FEF112311F40C94F408009162
:10112C002405109125051F3F09F40F3F10E009F429
:10113C001FEF112311F40C94A60810E00C94F50881
:10114C000091240510912505009326051093270581
:10115C00CF93DF9300912405109125051A930A93E0
:10116C000E94AE02DF91CF910093240510932505C8
:10117C0000912405109125051F3F09F40F3F10E045
:10118C0009F41FEF112311F40C94CF0810E00C9408
:10119C00F50800912405109125051F3F09F4073F20
:1011AC0010E009F41FEF112311F40C94E00810E087
:1011BC000C94F508CF93DF9300912405109125052D
:1011CC001A930A930E947804DF91CF910093200523
:1011DC001093210520932205309323051FEF0895CA
:1011EC00CF93DF93009120051091210520912205CA
:1011FC00309123053A932A931A930A93EBEDF1E07D
:10120C008F011A930A930E943E00DF91CF91EBED70
:10121C00F1E0EF93FF9310911F05012F112701505F
:10122C001040A0E2B0E0E89445F80E946537FF91C9
:10123C00EF91E00FF11F1191103010E009F01FEF4A
:10124C00089522970A811B8119830883CF93DF931A
:10125C00088119811A930A930E94AE02DF91CF91F3
:10126C001983088308811981103009F4003010E0CB
:10127C0009F41FEF112311F40C9446090C948809FE
:10128C000E944402EBEDF1E0EF93FF9300911A05FD
:10129C0010911B05000F111FFF91EF91E00FF11F33
:1012AC0010E000E0019311930E946402109102057A
:1012BC00123010E009F41FEF112311F40C947C0987
:1012CC000E944402EBEDF1E0EF93FF9300911A05BD
:1012DC0010911B05000F111FFF91EF91E00FF11FF3
:1012EC0010E000E0019311930E948402088119819F
:1012FC001F3F09F40F3F10E009F41FEF112311F405
:10130C000C942C0908952197E981FA81EF93FF93AE
:10131C00E2E3F2E7BF91AF91689444F80E94D136B2
:10132C0010E009F41FEF112311F40C94A00910E044
:10133C000C94230AE0EBF4E0EF93FF9310E2EBE064
:10134C00F0E0BF91AF913196319711F01D93FCCF26
:10135C001CE51F93E981FA81EF93FF9361E0FF9104
:10136C00EF910F910E947E3518831881103010E098
:10137C0009F41FEF112311F40C94F509E981FA819A
:10138C001081188318811B3010E011F008F01FEF4A
:10139C00112311F40C94D50910E00C94230AE98163
:1013AC00FA813196EF93FF93E0EBF4E0EF93FF9328
:1013BC001881012F1127FF91EF91DF01FF91EF9120
:1013CC0098010E940534E981FA81EF93FF9311E0B3
:1013DC001F93188170E00E942D340C94220A1881FE
:1013EC0011501B3010E011F008F01FEF112311F415
:1013FC000C94030A10E00C94230AE981FA813196CB
:10140C00EF93FF93E0EBF4E0EF93FF93188111500F
:10141C00012F1127FF91EF91DF01FF91EF919801BF
:10142C000E940534E981FA81EF93FF9311E01F9339
:10143C00188170E00E942D341FEF08952697CF93EA
:10144C00DF930E811F811A930A930E947804DF9117
:10145C00CF913B832A83198308833B812A8119818D
:10146C0008813F3F29F42F3F19F41F3F09F40F3F28
:10147C0010E009F41FEF112311F40C94480A10E04A
:10148C000C949C0AEBEDF1E0EF93FF9310E0E0E09D
:10149C00F2E0BF91AF913196319711F01D93FCCFD3
:1014AC0010E000E01D830C830C811D810F931F93B2
:1014BC0010911305012F112798011F910F911317EC
:1014CC0009F402171FEF08F01127112311F40C94E3
:1014DC009B0ACF93DF933B812A81198108810F935B
:1014EC001F932F933F930C811D8133272227FF914C
:1014FC00EF91BF91AF910A0F1B1F2E1F3F1F3A9305
:10150C002A931A930A93EBEDF1E08F011A930A9345
:10151C000E944100DF91CF91FE013496A081B181F0
:10152C001196A083B1830C945A0A1FEF0895249747
:10153C00E8E2F5E0319610E21193E8E2F5E0EF9382
:10154C00FF933196FA93EA9315E11A9317EF412220
:10155C001FEB4122EF81F8850E94AE3515E11F93F8
:10156C0018810F91011B102FFF91EF91108323967F
:10157C00E8E2F5E01081113010E011F008F01FEFF7
:10158C001F93E8E2F5E0EF93FF93E8E2F5E01081BA
:10159C00FF91EF91012F1127E00FF11F11911C35D5
:1015AC0010E009F41FEF0F911023112311F40C9488
:1015BC00ED0AE8E2F5E0EF93FF93E8E2F5E0108145
:1015CC001150FF91EF91153108F015E11193E8E2FC
:1015DC00F5E0319611911C3510E009F01FEF112345
:1015EC0011F40C94AA0CE8E2F5E0EF93FF93E2E31C
:1015FC00F2E7BF91AF91689444F80E94D13610E0A5
:10160C0009F41FEF112311F40C94290BE8E2F5E017
:10161C00EF93FF933196FA93EA9315E11A9317EF30
:10162C0041221FEB4122E1ECF4E00E94AE3515E1C2
:10163C001F9318810F91011B102FFF91EF911083B5
:10164C0023960C94AA0CE1ECF4E0EF93FF93E3E304
:10165C00F2E7BF91AF91689444F80E94D13610E044
:10166C0009F41FEF112311F40C94820BE8E2F5E05E
:10167C00EF93FF93E2E3F2E7BF91AF91689444F8E4
:10168C000E94D13610E009F01FEF1F93E8E2F5E05D
:10169C00319611911E3210E009F41FEF0F911023B7
:1016AC00112311F40C94660BE8E2F5E0EF93FF9331
:1016BC0011E01F9311E070E00E942D340C943C0B50
:1016CC00E8E2F5E0319611911C3510E009F01FEFBE
:1016DC00112311F40C94800BE3E3F2E7EF93FF93E7
:1016EC00E8E2F5E0EF93FF9315E11F9311E092E030
:1016FC000E9463340C94AA0C10E01B83E8E2F5E022
:10170C00EF93FF93E2E3F2E7BF91AF91689444F853
:10171C000E94D13610E009F01FEF1F93E8E2F5E0CC
:10172C00319611911E3210E009F41FEF0F91102326
:10173C00112311F40C94B00BE8E2F5E0EF93FF9356
:10174C0011E01F9311E070E00E942D341FEF1B83FA
:10175C000C94840B1B81112311F40C948E0CFE0140
:10176C003296FA93EA93EF93FF93E1ECF4E0108155
:10177C00FF91EF91108311E01A93108108810117EA
:10178C0010E011F008F01FEF112311F00C94ED0B89
:10179C00E1ECF4E0EF93FF931D81FF91EF91012FAA
:1017AC001127E00FF11F11911C3510E009F41FEF08
:1017BC00112311F40C94E40B0C94ED0BE981FA81D8
:1017CC0010811A9510831F3F11F00C94C40B2396B3
:1017DC001A8112301FEF08F01127112311F40C9409
:1017EC00260CE8E2F5E0EF93FF93E2E3F2E7BF911A
:1017FC00AF91689444F80E94D13610E009F41FEFC1
:10180C00112311F40C94240CE8E2F5E0EF93FF9310
:10181C003196FA93EA9315E11A9317EF41221FEBD5
:10182C0041221CE50E94F73615E11F9318810F9198
:10183C00011B102FFF91EF91108323960C948C0CAD
:10184C00FE01329610811A951083E8E2F5E01081C2
:10185C001F931A810F91100F1883FE013196FA9382
:10186C00EA9311E01083EF93FF931C81FF91EF91AA
:10187C001A931081088101171FEF08F0112711230B
:10188C0011F00C94600CE5E3F2E7EF93FF93E8E2C0
:10189C00F5E0EF93FF9315E11F9311E092E00E94A6
:1018AC006334E981FA81108113951083112311F0AF
:1018BC000C94400C2396E8E2F5E0EF93FF933196FD
:1018CC00FA93EA9315E11A9317EF41221FEB412289
:1018DC00E1ECF4E0EF93FF9311E01F931D810F9166
:1018EC00FF91EF910E94943515E11F9318810F9190
:1018FC00011B102FFF91EF9110832396E8E2F5E086
:10190C00EF93FF931881FF91EF9111930C94AA0C14
:10191C00E3E3F2E7EF93FF93E8E2F5E0EF93FF9355
:10192C0015E11F9311E092E00E946334E1ECF4E0C6
:10193C00EF93FF93E8E2F5E0EF93FF9315E11F932C
:10194C0011E090E00E946334E8E2F5E01081113080
:10195C0010E011F008F01FEF1F93E8E2F5E0EF93B1
:10196C00FF93E8E2F5E01081FF91EF91012F112731
:10197C00E00FF11F11911C3510E009F41FEF0F91CE
:10198C001023112311F40C94D90CE8E2F5E0EF9339
:10199C00FF93E8E2F5E010811150FF91EF911531C2
:1019AC0008F015E1119308952497E8E2F5E0EF9320
:1019BC00FF933196FA93EA9315E11A9317EF4122AC
:1019CC001FEB4122EF81F8850E94AE3515E11F9384
:1019DC0018810F91011B102FFF91EF91108323960B
:1019EC00E8E2F5E0EF93FF93E2E3F2E7BF91AF910A
:1019FC00689444F80E94D13610E009F41FEF1123CB
:101A0C0011F40C94170D0091BD041091BE0420919B
:101A1C00BF043091C0043B832A83198308830C9440
:101A2C005D0DE8E2F5E0319611911C3510E009F4FA
:101A3C001FEF112311F40C942F0D0091050510913B
:101A4C000605332722273B832A83198308830C94AA
:101A5C005D0DE8E2F5E0319611911E3210E009F4CB
:101A6C001FEF112311F40C94510D009105051091E9
:101A7C000605332722273B832A8319830883CF93B8
:101A8C00DF93EC81FD81FA93EA930E949D0ADF912A
:101A9C00CF910C945D0D0091BD041091BE0420916A
:101AAC00BF043091C0043B832A8319830883E8E286
:101ABC00F5E01081103010E011F008F01FEF1F93CB
:101ACC00E8E2F5E0319611911C3510E009F41FEFB6
:101ADC000F911023112311F40C947E0DE8E2F5E024
:101AEC00EF93FF9311E01F9311E070E00E942D34EF
:101AFC00E8E2F5E01081103010E011F008F01FEF73
:101B0C001F93E8E2F5E0EF93FF93E8E2F5E0108134
:101B1C00FF91EF91012F1127E00FF11F11911C354F
:101B2C0010E009F41FEF0F911023112311F40C9402
:101B3C00AD0DE8E2F5E0EF93FF93E8E2F5E01081FC
:101B4C001150FF91EF91153108F015E11193CF93DE
:101B5C00DF93E8E2F5E0FA93EA930E948909DF91BA
:101B6C00CF91112311F40C94540ECF93DF933B813E
:101B7C002A81198108813A932A931A930A930E9415
:101B8C008107DF91CF910E94F6081095112311F473
:101B9C000C94D60D00E010E020E030E00C94580ED0
:101BAC00EBEDF1E0EF93FF9310911F05012F11273F
:101BBC0001501040A0E2B0E0E89445F80E9465376F
:101BCC00FF91EF91E00FF11F3B9611911F9310E1E4
:101BDC000F91011710E009F41FEF112311F40C946D
:101BEC001D0ECF93DF93E0EBF4E0FA93EA93EBED69
:101BFC00F1E0EF93FF9310911F05012F1127015076
:101C0C001040A0E2B0E0E89445F80E946537FF91DF
:101C1C00EF91E00FF11FFA93EA930E941907DF91FD
:101C2C00CF91112311F40C941D0E0C942F0E0E94C5
:101C3C00DE071095112311F40C942A0E00E010E02D
:101C4C0020E030E00C94580E10E0112311F40C94A9
:101C5C00C90DCF93DF93EBEDF1E0EF93FF93109170
:101C6C001F05012F112701501040A0E2B0E0E894AD
:101C7C0045F80E946537FF91EF91E00FF11F7A96BE
:101C8C00019111911A930A930E947804DF91CF91DC
:101C9C003B832A83198308830C94AD0D3B812A81E5
:101CAC00198108810895E881F981FA93EA93E88112
:101CBC00F9813596EF93FF93E881F981B9960191FB
:101CCC001191FF91EF9101931193E881F981319674
:101CDC00EF93FF93CF93DF93E881F98135960191D0
:101CEC0011911A930A930E947804DF91CF91FF917E
:101CFC00EF910193119321933193E881F9813196FE
:101D0C0001911191219131913F3F29F42F3F19F409
:101D1C001F3F09F40F3F10E009F01FEF22960C94BF
:101D2C00980E22960895E881F981FA93EA93E88156
:101D3C00F9813196A081B18182819381119608F449
:101D4C000196A083B18382839383E881F9813196D4
:101D5C0001911191219131910F931F932F933F93E7
:101D6C000091090510910A053327222701501040D4
:101D7C00204030402095309510950095FF91EF91C3
:101D8C00BF91AF910A0F1B1F2E1F3F1F0F931F9365
:101D9C002F933F9310911305012F112733272227DF
:101DAC00E89445F80E9403388C019001507841F07A
:101DBC0001501040204030402095309510950095F2
:101DCC00303029F4203019F4103009F4003010E0D0
:101DDC0009F41FEF112311F40C94440FE881F981DD
:101DEC003596019111911F3F09F40F3F10E009F452
:101DFC001FEF112311F40C94070F10E022960C9492
:101E0C00490FE881F9813596EF93FF93CF93DF93D8
:101E1C00E881F9813596019111911A930A930E94E8
:101E2C00AE02DF91CF91FF91EF9101931193E88175
:101E3C00F9813596019111911F3F09F40F3F10E084
:101E4C0009F01FEF112311F40C94440FE881F98170
:101E5C003196EF93FF93CF93DF93E881F981359619
:101E6C00019111911A930A930E947804DF91CF91FA
:101E7C00FF91EF9101931193219331931FEF2296D0
:101E8C000C94490F229608952297EA81FB81FA93CC
:101E9C00EA93E881F9813196A081B18182819381A5
:101EAC00119608F40196A083B18382839383E88111
:101EBC00F981319601911191219131910F931F93D9
:101ECC002F933F930091090510910A053327222780
:101EDC0001501040204030402095309510950095D1
:101EEC00FF91EF91BF91AF910A0F1B1F2E1F3F1F48
:101EFC000F931F932F933F9310911305012F1127CD
:101F0C0033272227E89445F80E9403388C0190016E
:101F1C00507841F0015010402040304020953095D1
:101F2C0010950095303029F4203019F4103009F454
:101F3C00003010E009F41FEF112311F40C941B1066
:101F4C00E881F9813596019111911B830A83E8810F
:101F5C00F9813596EF93FF930E943E03FF91EF9129
:101F6C0001931193E881F9813596019111911F3FED
:101F7C0009F40F3F10E009F41FEF112311F40C9436
:101F8C00CB0F10E022960C942010CF93DF930A8194
:101F9C001B811A930A93EA81FB8135960191119169
:101FAC001A930A930E94EC02DF91CF91CF93DF93A7
:101FBC00E881F9813596019111911A930A931FEFDB
:101FCC000FEF1A930A930E94EC02DF91CF91E881F4
:101FDC00F9813196EF93FF93CF93DF93E881F981E9
:101FEC003596019111911A930A930E947804DF910E
:101FFC00CF91FF91EF910193119321933193CF9353
:10200C00DF93E881F9813196019111912191319100
:10201C003A932A931A930A93EBEDF1E08F011A93FA
:10202C000A930E943E00DF91CF911FEF22960C94F1
:10203C00201022960895E881F981FA93EA93CF93C0
:10204C00DF93E881F981BF96019111912191319132
:10205C003A932A931A930A930E948107DF91CF91A6
:10206C000E94F6081095112311F40C94421010E004
:10207C0000E022960C94C310EBEDF1E0EF93FF938C
:10208C0010911F05012F112701501040A0E2B0E064
:10209C00E89445F80E946537FF91EF91E00FF11F2E
:1020AC003B9611911F9310E10F91011710E009F06D
:1020BC001FEF112311F40C948A10CF93DF93E88156
:1020CC00F9813F96FA93EA93EBEDF1E0EF93FF93EE
:1020DC0010911F05012F112701501040A0E2B0E014
:1020EC00E89445F80E946537FF91EF91E00FF11FDE
:1020FC00FA93EA930E941907DF91CF91112311F4FF
:10210C000C948A100C949B100E94DE0710951123DE
:10211C0011F40C94961010E000E022960C94C3106D
:10212C0010E0112311F40C943610E881F9813F96DC
:10213C00EF93FF93EBEDF1E0EF93FF9310911F05FD
:10214C00012F112701501040A0E2B0E0E89445F8AF
:10215C000E946537FF91EF91E00FF11FBF91AF9196
:10216C0020E230E00E940534E881F981B9960191B2
:10217C00119122960C94C3102296089510911F056C
:10218C00113010E009F41FEF112311F40C94D3104B
:10219C001FEF0C94FC100C94FB10EBEDF1E0EF93A3
:1021AC00FF9310911F051150012F11270150104062
:1021BC00A0E2B0E0E89445F80E946537FF91EF91FA
:1021CC00E00FF11F3B9611911F931FE00F91011728
:1021DC0010E009F41FEF112311F40C94FB1017E01D
:1021EC001093DA0110E00C94FC101FEF08950E947C
:1021FC007D3308950E949F330895E881F981FA9305
:10220C00EA93E881F9817A9611911F9310E10F916D
:10221C00011710E009F41FEF112311F40C941A119B
:10222C0010E022960C946113CF93DF93E881F9812F
:10223C00BF9601911191219131913A932A931A935E
:10224C000A930E948107DF91CF910E94F608112317
:10225C0011F40C940312EBEDF1E0EF93FF9310915A
:10226C001F05012F112701501040A0E2B0E0E894A7
:10227C0045F80E946537FF91EF91E00FF11F3B96F7
:10228C001191107110311FEF09F010E0109511230E
:10229C0011F40C94F811CF93DF93E881F9813F96F8
:1022AC00FA93EA93EBEDF1E0EF93FF9310911F0596
:1022BC00012F112701501040A0E2B0E0E89445F83E
:1022CC000E946537FF91EF91E00FF11FFA93EA93AB
:1022DC000E941907DF91CF91112311F40C94F8117E
:1022EC00EBEDF1E0EF93FF9310911F05012F1127F8
:1022FC0001501040A0E2B0E0E89445F80E94653728
:10230C00FF91EF91E00FF11F3B961191117011307D
:10231C001FEF09F010E0112311F40C949C1117E03D
:10232C001093DA0110E022960C9461130E94C410F1
:10233C001095112311F40C94A71110E022960C9413
:10234C006113CF93DF93009120051091210520910B
:10235C002205309123053A932A931A930A93EBEDB5
:10236C00F1E08F011A930A930E943E00DF91CF9106
:10237C00EBEDF1E0EF93FF9310911F05012F112767
:10238C0001501040A0E2B0E0E89445F80E94653797
:10239C00FF91EF91E00FF11FEF93FF93E881F9812B
:1023AC003F96BF91AF9120E230E00E940534CF936D
:1023BC00DF93009120051091210520912205309189
:1023CC0023053A932A931A930A93EBEDF1E08F01CC
:1023DC001A930A930E944100DF91CF911FEF22962E
:1023EC000C9461130E94DE071095112311F40C94C8
:1023FC0001120C9403120C942B11CF93DF93E881F0
:10240C00F981BF9601911191219131913A932A93BF
:10241C001A930A930E948107DF91CF910E94F608CC
:10242C00112311F40C940F13EBEDF1E0EF93FF93E8
:10243C0010911F05012F112701501040A0E2B0E0B0
:10244C00E89445F80E946537FF91EF91E00FF11F7A
:10245C001191153011F0153E01F010E009F41FEF49
:10246C00112311F40C947412EBEDF1E0EF93FF9344
:10247C0010911F05012F112701501040A0E2B0E070
:10248C00E89445F80E946537FF91EF91E00FF11F3A
:10249C00EF93FF93E881F9813F96BF91AF9120E2D2
:1024AC0030E00E940534CF93DF930091200510910A
:1024BC00210520912205309123053A932A931A93F2
:1024CC000A93EBEDF1E08F011A930A930E944100FD
:1024DC00DF91CF911FEF22960C9461130E94DE07BF
:1024EC001095112311F40C940D1310911E0511234A
:1024FC0011F40C94851210E022960C946113009147
:10250C002405109125051F3F09F4073F10E009F43D
:10251C001FEF112311F40C94971210E022960C94D7
:10252C00611300912405109125051F3F09F40F3FFD
:10253C0010E009F41FEF112311F40C940D130E94F9
:10254C003E0300932405109325050091240510915A
:10255C0025051F3F09F40F3F10E009F41FEF11236D
:10256C0011F40C94BD1210E022960C946113CF93CD
:10257C00DF9300912405109125051A930A930E946C
:10258C00240ADF91CF911095112311F40C94D212DF
:10259C0010E022960C946113CF93DF9300912605E3
:1025AC00109127051A930A93009124051091250583
:1025BC001A930A930E94EC02DF91CF91CF93DF9391
:1025CC0000912405109125051A930A931FEF0FEF24
:1025DC001A930A930E94EC02DF91CF91CF93DF9371
:1025EC0000912405109125051A930A930E947804F2
:1025FC00DF91CF91009320051093210520932205A4
:10260C003093230511E010931F050C940F130C94B9
:10261C001412CF93DF930091200510912105209186
:10262C002205309123053A932A931A930A93EBEDE2
:10263C00F1E08F011A930A930E943E00DF91CF9133
:10264C00EBEDF1E0EF93FF9310911F05012F112794
:10265C0001501040A0E2B0E0E89445F80E946537C4
:10266C00FF91EF91E00FF11FEF93FF93E881F98158
:10267C003F96BF91AF9120E230E00E940534CF939A
:10268C00DF930091200510912105209122053091B6
:10269C0023053A932A931A930A93EBEDF1E08F01F9
:1026AC001A930A930E944100DF91CF911FEF22965B
:1026BC000C94611322960895EA81FB81F3960191A3
:1026CC001191103011F00C947113003011F00C9426
:1026DC0071130C947913103011F00C947F1301309A
:1026EC0011F00C947F13088119810C94C2130C9473
:1026FC00C213103011F00C948F13023011F00C94A3
:10270C008F1308811981169507950C94C2130C949C
:10271C00C213103011F00C94A013043011F00C946F
:10272C00A0130881198122E00E9455380C94C21321
:10273C000C94C213103011F00C94B113083011F03A
:10274C000C94B1130881198123E00E9455380C9424
:10275C00C2130C94C213088119810F931F93EA8141
:10276C00FB81F39601911191E89445F8BF91AF91DB
:10277C000E9486370C94C21308952297EC81FD8138
:10278C00F39601911191198308830A811B811030F2
:10279C0011F00C94DB13003011F00C94DB1310E0EF
:1027AC0000E00C9429140C942914103011F00C94A2
:1027BC00E913013011F00C94E913088119810C9480
:1027CC0029140C942914103011F00C94F9130230C4
:1027DC0011F00C94F91308811981000F111F0C943E
:1027EC0029140C942914103011F00C940A14043090
:1027FC0011F00C940A140881198122E00E9471389E
:10280C000C9429140C942914103011F00C941B14F2
:10281C00083011F00C941B140881198123E00E94DC
:10282C0071380C9429140C942914088119810F9374
:10283C001F930A811B81E89445F8BF91AF910E94C8
:10284C0065370C9429140895EC81FD81F396019160
:10285C001191103011F00C943F14003011F00C94C5
:10286C003F1400E010E020E030E00C949E140C9437
:10287C009E14103011F00C944F14013011F00C9484
:10288C004F143B812A81198108810C949E140C945D
:10289C009E14103011F00C946314023011F00C944F
:1028AC0063143B812A8119810881369527951795E8
:1028BC0007950C949E140C949E14103011F00C94EB
:1028CC007614043011F00C9476143B812A81198112
:1028DC000881E2E00E9461380C949E140C949E14C2
:1028EC00103011F00C948914083011F00C948914E8
:1028FC003B812A8119810881E3E00E9461380C94A4
:10290C009E140C949E143B812A81198108810F938B
:10291C001F932F933F93EC81FD81F39601911191BD
:10292C0033272227E89445F80E9403380C949E1410
:10293C0008952497E885F985F39601911191332731
:10294C0022273B832A83198308833F812E811D8193
:10295C000C81303029F4203019F4103009F4003097
:10296C0010E009F41FEF112311F40C94C51400E0CE
:10297C0010E020E030E00C9449150C9449153F818F
:10298C002E811D810C81303029F4203019F4103047
:10299C0009F4013010E009F41FEF112311F40C9429
:1029AC00DF143B812A81198108810C9449150C9400
:1029BC0049153F812E811D810C81303029F4203046
:1029CC0019F4103009F4023010E009F41FEF112350
:1029DC0011F40C94FD143B812A8119810881000F9C
:1029EC00111F221F331F0C9449150C9449153F815C
:1029FC002E811D810C81303029F4203019F41030D7
:102A0C0009F4043010E009F41FEF112311F40C94B5
:102A1C001A153B812A8119810881E2E00E947D38D8
:102A2C000C9449150C9449153F812E811D810C8104
:102A3C00303029F4203019F4103009F4083010E04B
:102A4C0009F41FEF112311F40C9437153B812A81E3
:102A5C0019810881E3E00E947D380C9449150C948F
:102A6C0049153B812A81198108810F931F932F935C
:102A7C003F933F812E811D810C81E89445F80E9483
:102A8C00B6370C94491508952297FE01EF93FF93E6
:102A9C000E94FD10FF91EF9101931193E881F98150
:102AAC008F01103009F4003010E009F41FEF1123EE
:102ABC0011F40C94641510E00C94F615E881F9816E
:102ACC0011E01193E881F981BF96EF93FF93CF93B7
:102ADC00DF93FE013F96FA93EA930E94DA0CDF91A2
:102AEC00CF91FF91EF910193119321933193E88151
:102AFC00F981F3960091D8011091D90101931193AA
:102B0C00E881F981BF960191119121913191303079
:102B1C0029F4203019F4103009F4003010E009F4D5
:102B2C001FEF112311F40C94A915CF93DF93088197
:102B3C001981F8011A930A930E940011DF91CF9129
:102B4C0010E00C94F615CF93DF9310E01A932D97A9
:102B5C004F92FE01EF93FF933196FA93EA931CE0A8
:102B6C001A9317EF41221FEB4122FE0173960E942C
:102B7C00AE351CE01F9318810F91011B102FFF9194
:102B8C00EF91108323964F90EE85FF853F96FA9335
:102B9C00EA930E94A605DF91CF911095112311F4B1
:102BAC000C94E615CF93DF9308811981F8011A93E1
:102BBC000A930E940011DF91CF9110E00C94F6154E
:102BCC00A5E2B0E0AC0FBD1FED91FD91EF93FF932B
:102BDC0008811981F801FF91EF91019311931FEF77
:102BEC000895249700E010E020E030E0EC81FD81B6
:102BFC000193119321933193CF93DF9310E01A93A8
:102C0C002D974F92FE01EF93FF933196FA93EA932F
:102C1C001CE01A9317EF41221FEB4122FE0177961D
:102C2C000E94AE351CE01F9318810F91011B102FD1
:102C3C00FF91EF91108323964F90E0EBF4E0FA9321
:102C4C00EA930E94A605DF91CF911095112311F400
:102C5C000C94331610E00C949616CF93DF93669772
:102C6C004F92FE01EF93FF933196FA93EA9315E19D
:102C7C001A9317EF41221FEB4122FE01BC960E94D2
:102C8C00AE3515E11F9318810F91011B102FFF9189
:102C9C00EF91108323964F902D974F92FE01EF9357
:102CAC00FF933196FA93EA931CE01A9317EF4122A3
:102CBC001FEB4122FE01BC960E94AE351CE01F9317
:102CCC0018810F91011B102FFF91EF911083239608
:102CDC004F9017E21A93EBEDF3E0FA93EA930E940C
:102CEC009716DF91CF911095112311F40C94861641
:102CFC0019E01093DA0110E00C9496160C949616C9
:102D0C00EBEDF3E0B9960191119121913191EC81A8
:102D1C00FD8101931193219331931FEF0C9496161F
:102D2C0008952497EC81FD81FA93EA93E881F98167
:102D3C00BD96EF93FF93FE0138961191FF91EF91A1
:102D4C001193E881F981F996EF93FF93CF93DF9379
:102D5C00FE017696FA93EA930E94DA0CDF91CF91FA
:102D6C00FF91EF910193119321933193CF93DF93C3
:102D7C001FEF1A932D974F92FE01EF93FF9331960D
:102D8C00FA93EA931CE01A9317EF41221FEB4122AE
:102D9C00FE017A960E94AE351CE01F9318810F91AC
:102DAC00011B102FFF91EF91108323964F90EE850E
:102DBC00FF85BE96FA93EA930E94A605DF91CF9108
:102DCC001095112311F40C94EF1610E022960C942C
:102DDC003318CF93DF93E881F981F9960191119122
:102DEC00219131913A932A931A930A930E94810765
:102DFC00DF91CF910E94F6081095112311F40C94D9
:102E0C000B1710E022960C943318EBEDF1E0EF93D6
:102E1C00FF9310911F05012F112701501040A0E2C4
:102E2C00B0E0E89445F80E946537FF91EF91E00F10
:102E3C00F11F1191153021F01E3211F0153E01F0E9
:102E4C0010E009F41FEF1095112311F40C942718BE
:102E5C00EBEDF1E0EF93FF9310911F05012F11277C
:102E6C0001501040A0E2B0E0E89445F80E946537AC
:102E7C00FF91EF91E00FF11F3B9611911F93FE0113
:102E8C00389611910F911023011710E009F41FEFE0
:102E9C001F93EBEDF1E0EF93FF9310911F05012FC2
:102EAC00112701501040A0E2B0E0E89445F80E94D0
:102EBC006537FF91EF91E00FF11F7496019111911D
:102ECC00103009F4003010E009F41FEF0F911023BB
:102EDC00112311F40C942718CF93DF93E881F98117
:102EEC00BE96FA93EA93EBEDF1E0EF93FF9310911A
:102EFC001F05012F112701501040A0E2B0E0E8940B
:102F0C0045F80E946537FF91EF91E00FF11FFA939E
:102F1C00EA930E941907DF91CF91112311F40C94BD
:102F2C002718EBEDF1E0EF93FF9310911F05012FA4
:102F3C00112701501040A0E2B0E0E89445F80E943F
:102F4C006537FF91EF91E00FF11FEF93FF93E8814D
:102F5C00F9813D96EF93FF93FF91EF91DF01FF9184
:102F6C00EF9120E230E00E940534CF93DF93E881AB
:102F7C00F9813D96A09720E230E0DE010E940534F5
:102F8C00A0E2B0E0AC0FBD1FED91FD91FA93EA9376
:102F9C000E94CB04DF91CF91E881F981EB5BFF4F6D
:102FAC0010911F051193E881F981EA5BFF4F0091A5
:102FBC001C0510911D0501931193E881F981EF5BBC
:102FCC00FF4FEF93FF930091200510912105209165
:102FDC00220530912305FF91EF91019311932193D9
:102FEC003193E881F981E85BFF4F10911E05119335
:102FFC00E881F981FF960091240510912505019334
:10300C001193E881F981FD96009126051091270511
:10301C00019311930E94C4101095112311F40C9478
:10302C002318E881F9817896EF93FF9311E0012F33
:10303C00FF91EF911081102B10831FEF22960C94AF
:10304C0033180E94DE071095112311F40C9400170D
:10305C0010E022960C94331822960895E881F98199
:10306C00FA93EA93E881F981EB5BFF4F119110938E
:10307C001F05E881F981EA5BFF4F019111910093E3
:10308C001C0510931D05E881F981EF5BFF4F019141
:10309C0011912191319100932005109321052093DA
:1030AC00220530932305E881F981E85BFF4F1191EC
:1030BC0010931E05E881F981FF96019111910093FF
:1030CC00240510932505E881F981FD960191119154
:1030DC0000932605109327050E94DE07112311F497
:1030EC000C94A2190E94F6081095112311F40C945B
:1030FC00831810E022960C94A419EBEDF1E0EF93F9
:10310C00FF9310911F05012F112701501040A0E2D1
:10311C00B0E0E89445F80E946537FF91EF91E00F1D
:10312C00F11F1191153021F01E3211F0153E01F0F6
:10313C0010E009F41FEF1095112311F40C94A01951
:10314C00EBEDF1E0EF93FF9310911F05012F112789
:10315C0001501040A0E2B0E0E89445F80E946537B9
:10316C00FF91EF91E00FF11F3B9611911F93E881B6
:10317C00F981BD9611910F911023011710E009F4FC
:10318C001FEF1F93EBEDF1E0EF93FF9310911F05F1
:10319C00012F112701501040A0E2B0E0E89445F84F
:1031AC000E946537FF91EF91E00FF11F749601912A
:1031BC001191103009F4003010E009F41FEF0F9159
:1031CC001023112311F40C94A019CF93DF93E881F1
:1031DC00F981BE96FA93EA93EBEDF1E0EF93FF934E
:1031EC0010911F05012F112701501040A0E2B0E0F3
:1031FC00E89445F80E946537FF91EF91E00FF11FBD
:10320C00FA93EA930E941907DF91CF91112311F4DD
:10321C000C94A019EBEDF1E0EF93FF9310911F05C7
:10322C00012F112701501040A0E2B0E0E89445F8BE
:10323C000E946537FF91EF91E00FF11FEF93FF9321
:10324C00E881F9813D96EF93FF93FF91EF91DF01B8
:10325C00FF91EF9120E230E00E940534CF93DF9391
:10326C00E881F9813D96A09720E230E0DE010E94D2
:10327C000534A0E2B0E0AC0FBD1FED91FD91FA93C7
:10328C00EA930E94CB04DF91CF91E881F981EB5B4B
:10329C00FF4F10911F051193E881F981EA5BFF4FF5
:1032AC0000911C0510911D0501931193E881F98182
:1032BC00EF5BFF4FEF93FF930091200510912105D9
:1032CC002091220530912305FF91EF9101931193E9
:1032DC0021933193E881F981E85BFF4F10911E0532
:1032EC001193E881F981FF96009124051091250531
:1032FC0001931193E881F981FD96009126051091B7
:10330C002705019311930E94C4101095112311F4F9
:10331C000C949C19E881F9817896EF93FF9311E056
:10332C00012FFF91EF911081102B10831FEF22962C
:10333C000C94A4190C947218229610E00895CF9353
:10334C00DF93FE01019111911A930A930E94B333FA
:10335C00DF91CF911095112311F40C94B81910E052
:10336C000C942B1AE881F981FA93EA93E881F9819C
:10337C001191113011F0123001F010E009F41FEF2F
:10338C001095112311F40C94CF1910E022960C9483
:10339C002B1AE881F9813596EF93FF93CF93DF9346
:1033AC000A811B81F8011A930A930E942110DF9164
:1033BC00CF91FF91EF9101931193E881F9813596AB
:1033CC0001911191103009F4003010E009F41FEF55
:1033DC00112311F40C94F61910E022960C942B1A6C
:1033EC00CF93DF930A811B811A930A930E94590E83
:1033FC00DF91CF911095112311F40C94091A10E060
:10340C0022960C942B1AE881F981379610E000E093
:10341C0001931193E881F9813B9600E010E020E0E4
:10342C0030E00193119321933193E881F98139961E
:10343C0010E000E001931193E881F98112E01193FF
:10344C001FEF22960C942B1A229608952297FE01B8
:10345C00EF93FF93EA81FB8101911191FF91EF9121
:10346C0001931193EA81FB8110E000E00193119329
:10347C00CF93DF93FE01019111911A930A930E944D
:10348C00B333DF91CF911095112311F40C94511A91
:10349C0010E00C94BC1AE881F981FA93EA93E88164
:1034AC00F9811191103011F00C945E1A0C94621A7F
:1034BC00113011F00C94731ACF93DF930A811B8196
:1034CC00F8011A930A930E940011DF91CF9110E03A
:1034DC0022960C94BC1A0C94AF1A133011F00C9465
:1034EC00791A0C947D1A143011F00C94AF1AE881EF
:1034FC00F981BB96EF93FF93E881F9813B9601919B
:10350C00119121913191FF91EF910193119321939D
:10351C003193CF93DF930A811B811A930A930E94F4
:10352C000311DF91CF911095112311F40C94AD1A66
:10353C00CF93DF930A811B81F8011A930A930E949F
:10354C000011DF91CF9110E022960C94BC1A0C94D0
:10355C00AF1A2296CF93DF9308811981F8011A9341
:10356C000A930E940011DF91CF911FEF0895CF9322
:10357C00DF93FE01019111911A930A930E94B333C8
:10358C00DF91CF911095112311F40C94D01A1FEFE9
:10359C000C940A1BE881F981FA93EA93E881F9818A
:1035AC001191123010E009F01FEF112311F40C945B
:1035BC00E31A10E022960C940A1BE881F981BB9661
:1035CC0001911191219131910F931F932F933F935F
:1035DC00E881F9813B960191119121913191D801AA
:1035EC00F9013F912F911F910F913F1729F42E173D
:1035FC0019F41B1709F40A171FEF10F009F0112723
:10360C0022960C940A1B229608952497CF93DF934D
:10361C00FE013A96019111911A930A930E94B333C9
:10362C00DF91CF911095112311F40C94261B10E00F
:10363C0000E0EC81FD810193119310E00C944B1E82
:10364C00CF93DF930A851B85F8011A930A9308859B
:10365C0019851A930A930E94C313DF91CF911F838C
:10366C000E83EA85FB85FA93EA93E881F98111913F
:10367C00123010E009F01FEF112311F40C944A1BC7
:10368C0010E022960C944B1EE881F981399610E0DB
:10369C0000E00193119310E000E0EE81FF810193B3
:1036AC001193E881F9813B9601911191219131910E
:1036BC000F931F932F933F93E881F981BB96019150
:1036CC00119121913191D801F9013F912F911F91C5
:1036DC000F913F1729F42E1719F41B1709F40A1729
:1036EC0010E008F01FEF112311F40C94811B10E073
:1036FC0022960C944B1EE881F981BB960191119195
:10370C00219131910F931F932F933F93E881F9816E
:10371C003B96019111912191319101501040204023
:10372C0030402095309510950095FF91EF91BF9109
:10373C00AF910A0F1B1F2E1F3F1F0F931F932F9329
:10374C003F930885198533272227D801F9013F912A
:10375C002F911F910F913F1729F42E1719F41B1756
:10376C0009F40A171FEF08F01127112311F40C9418
:10377C00E31BE881F981BB96019111912191319163
:10378C000F931F932F933F93E881F9813B960191FF
:10379C0011912191319101501040204030402095E1
:1037AC00309510950095FF91EF91BF91AF910A0F55
:1037BC001B1F2E1F3F1F198708870885198510307E
:1037CC0009F4003010E011F008F01FEF112311F490
:1037DC000C94311EE881F9813796019111910F9368
:1037EC001F93088519853F912F91020F131F1D837D
:1037FC000C830C811D810F931F9300910B0510916D
:10380C000C0598011F910F91131709F402171FEF64
:10381C0008F01127112311F40C94A01CCF93DF9303
:10382C00EC85FD85319601911191219131913A935D
:10383C002A931A930A93EBEDF1E08F011A930A93F2
:10384C000E943E00DF91CF91EBEDF1E0EF93FF93FF
:10385C00E881F981379601911191FF91EF91E00F79
:10386C00F11FEF93FF930A851B850F931F93E8813C
:10387C00F9813996019111913F912F91020F131FEC
:10388C000F931F9308851985FF91EF91DF01FF912D
:10389C00EF9198010E940534E881F9813796EF93F6
:1038AC00FF930C811D81FF91EF9101931193EE8198
:1038BC00FF81EF93FF9308851985B801FF91EF9174
:1038CC00A081B181A60FB71FA083B183E881F981D4
:1038DC003B96EF93FF930885198533272227B80170
:1038EC00C901FF91EF9120813181A281B381260F13
:1038FC00371FA81FB91F20833183A283B383CF93B3
:10390C00DF930C851D85F8011A930A93E885F985D8
:10391C00008111811A930A930E946213DF91CF9157
:10392C00EE81FF81019311931FEF22960C944B1E95
:10393C000C942F1E0C811D810F931F9300910B056E
:10394C0010910C0598011F910F91131709F4021790
:10395C0010E009F41FEF112311F40C94501DCF93B8
:10396C00DF93EC85FD853196019111912191319177
:10397C003A932A931A930A93EBEDF1E08F011A9381
:10398C000A930E943E00DF91CF91EBEDF1E0EF93B3
:10399C00FF93E881F981379601911191FF91EF9195
:1039AC00E00FF11FEF93FF930A851B850F931F9375
:1039BC00E881F9813996019111913F912F91020F74
:1039CC00131F0F931F9308851985FF91EF91DF014A
:1039DC00FF91EF9198010E940534CF93DF930C85F2
:1039EC001D851A930A930E94990EDF91CF91109521
:1039FC00112311F40C94061D10E022960C944B1E0E
:103A0C00E881F981379610E000E001931193EE8183
:103A1C00FF81EF93FF9308851985B801FF91EF9112
:103A2C00A081B181A60FB71FA083B183E881F98172
:103A3C003B96EF93FF930885198533272227B8010E
:103A4C00C901FF91EF9120813181A281B381260FB1
:103A5C00371FA81FB91F20833183A283B383CF9351
:103A6C00DF930C851D85F8011A930A93E885F98577
:103A7C00008111811A930A930E946213DF91CF91F6
:103A8C00EE81FF81019311931FEF22960C944B1E34
:103A9C000C942F1E0C811D810F931F9300910B050D
:103AAC0010910C0598011F910F91131709F402172F
:103ABC0010E011F008F01FEF112311F40C942F1EDD
:103ACC0000910B0510910C050F931F93E881F98160
:103ADC00379601911191019509F41A9510953F9122
:103AEC002F91020F131F1B830A83CF93DF93EC8557
:103AFC00FD85319601911191219131913A932A933F
:103B0C001A930A93EBEDF1E08F011A930A930E943A
:103B1C003E00DF91CF91EBEDF1E0EF93FF93E88165
:103B2C00F981379601911191FF91EF91E00FF11FFF
:103B3C00EF93FF930A851B850F931F93E881F981FF
:103B4C003996019111913F912F91020F131F0F93F1
:103B5C001F930A811B81FF91EF91DF01FF91EF9180
:103B6C0098010E940534CF93DF930C851D851A9321
:103B7C000A930E94990EDF91CF911095112311F4A5
:103B8C000C94E11DCF93DF930C851D85F8011A93DE
:103B9C000A93E885F985008111811A930A930E9492
:103BAC006213DF91CF91EE81FF810193119310E0AD
:103BBC0022960C944B1EE881F981379610E000E0B8
:103BCC0001931193FE013896EF93FF930A811B81A9
:103BDC00B801FF91EF91A081B181A61BB70BA08317
:103BEC00B183E881F9813996EF93FF930A811B81A8
:103BFC00B801FF91EF91A081B181A60FB71FA083EF
:103C0C00B183E881F9813B96EF93FF930A811B8185
:103C1C0033272227B801C901FF91EF91208131810F
:103C2C00A281B381260F371FA81FB91F20833183B0
:103C3C00A283B383EE81FF81EF93FF930A811B81F3
:103C4C00B801FF91EF91A081B181A60FB71FA0839E
:103C5C00B1830C94E31BCF93DF930C851D85F80186
:103C6C001A930A93E885F985008111811A930A93B6
:103C7C000E946213DF91CF91EE81FF81019311932A
:0C3C8C001FEF22960C944B1E2296089508
:10FC0000EEEFFDE71591153529F415911A3A11F427
:10FC10000C9400000E942F7E08953D9A459818E1AB
:10FC20001093C10017E21093C40010E01093C500B8
:10FC30001EE01093C20008951091C00017FFFCCF82
:10FC40001091C60008951F931091C00015FFFCCFBE
:10FC50001F911093C60008950C9400000895F89425
:10FC6000442410E10FEF1EBF0DBFCFEBD0E1D5DF75
:10FC7000E3DF1F3321F416E4E6DF14E431C011346E
:10FC800009F43EC0193409F42DC0183521F411E1EE
:10FC900017BFE895E1CF143409F454C0153409F4C2
:10FCA0003AC0103509F459C0123509F473C015353E
:10FCB00009F47DC0123409F485C0133409F491C0ED
:10FCC000103711F416E40CC0173509F42CC019369E
:10FCD00021F415EEB8DF17E203C01FE301C01DE0F9
:10FCE000B2DFC6CF19E4AFDF1EE1ADDF16E9ABDF4F
:10FCF00019E0A9DF10E8A7DF10E0A5DF1EE7F0CFCD
:10FD00009BDF1F9399DF0F91000F111F10937C0F42
:10FD100000937B0FE4CF43E0F0917C0FE0917B0FE9
:10FD2000E0706BD0DCCF88DF1F9386DF0F91000F70
:10FD3000EDE7FFE01127E00FF11F7EDF11937CDF7D
:10FD40001193CDCF00E02227EDE7FFE075DF11939F
:10FD5000210F0A95D9F7122FC3CF20E8ADE7BFE0F6
:10FD6000F0917C0FE0917B0FE0700D901D9041E0D1
:10FD700044D032962A95C9F711271A95F1F745E034
:10FD8000F0917C0FE0917B0FE07037D011271A952E
:10FD9000F1F7A5CFF0917C0FE0917B0FADE7BFE0CD
:10FDA00000E0C8950D9231960A95D9F798CFADE746
:10FDB000BFE030E022271D91210F45DF3A95D9F7AA
:10FDC000122F8ECF39DFE12F37DFF12F35DFF99991
:10FDD000FECFE1BDF2BDF89A000010BDFA9AF99A83
:10FDE0007ECF2ADFE12F28DFF12FF999FECFE1BD89
:10FDF000F2BDF89A000010B573CF47BFE895000038
:10FE000001C00000F999FECF57B750FDFBCF089510
:103C98003D9A459A399A10EF12B910EF1BB9409A1C
:103CA800469A0895E0E0F0E00E94243410933B0621
:103CB80010E010933D0610E000E0009339061093E1
:103CC8003A06089541980895419A0895619710E039
:103CD8001883FE013196EF93FF933196FA93EA9396
:103CE80016E01A9317EF41221FEB41220C891D8918
:103CF8000F931F9310E01F9310E01F9310E21F9380
:103D0800E89445F80E94403616E01F9318810F91F9
:103D1800011B102FFF91EF9110832396FE01389617
:103D2800EF93FF933196FA93EA9318E01A9317EFFB
:103D380041221FEB4122FE013496EF93FF9314E0DA
:103D48001F9310E31A931F91FF91EF91EF93FF9345
:103D58000981101708F0102F0191F991101B38F004
:103D680031F0E12F1F2F0E94F736EA95E1F7102F67
:103D780021E02F930F91FF91EF910E949435EAE390
:103D8800F2E7B591BB2311F00E94A83518E01F9304
:103D980018810F91011B102FFF91EF91108323962B
:103DA800CF93DF9366974F92FE01EF93FF9331967F
:103DB800FA93EA9315E11A9317EF41221FEB412278
:103DC8001CE50E94F73615E11F9318810F91011B1E
:103DD800102FFF91EF91108323964F902D974F92BC
:103DE800FE01EF93FF933196FA93EA931CE01A933E
:103DF80017EF41221FEB4122FE01BE960E94AE350D
:103E08001CE01F9318810F91011B102FFF91EF9158
:103E1800108323964F9017E21A93E0E8F5E0FA939F
:103E2800EA930E949716DF91CF91112311F40C9415
:103E38008E1F09891A890093390610933A06E8E219
:103E4800F6E0EF93FF933196FA93EA931CE01A9306
:103E580017EF41221FEB4122E0E8F5E00E94AE3562
:103E68001CE01F9318810F91011B102FFF91EF91F8
:103E780010832396CF93DF9366974F92FE01EF93BB
:103E8800FF933196FA93EA9315E11A9317EF4122BB
:103E98001FEB41221CE50E94F73615E11F9318819C
:103EA8000F91011B102FFF91EF91108323964F90D4
:103EB8002D974F92FE01EF93FF933196FA93EA9371
:103EC8001CE01A9317EF41221FEB4122E0E8F5E0CE
:103ED8000E94AE351CE01F9318810F91011B102F13
:103EE800FF91EF91108323964F90E8E2F6E03D961C
:103EF800FA93EA930E94F715DF91CF91CF93DF935E
:103F0800EEE7F5E0FA93EA930E942C1ADF91CF913D
:103F18001FEF18831881089521970E941032188383
:103F28001881112311F40C949B1F0C949E1F10E010
:103F38000C94BB1FCF93DF930E944400DF91CF9175
:103F480018831881112311F40C94AC1F0C94AF1F23
:103F580010E00C94BB1F0E941D32112311F40C9425
:103F6800B71F0C94BA1F10E00C94BB1F1FEF0895E5
:103F78000DB5112707FD1FEF112311F40C94BC1F79
:103F880008950DB5112707FD1FEF112311F40C94A7
:103F9800C51F18811EBD0895289813E01EBD0DB5D4
:103FA800112707FD1FEF112311F40C94D31F1C8157
:103FB8001EBD0DB5112707FD1FEF112311F40C9439
:103FC800DD1F0A811B81103009F4003010E011F068
:103FD80008F01FEF112311F40C941E20FE013296F5
:103FE800A081B1811197A083B18310E01EBD0DB5EA
:103FF800112707FD1FEF112311F40C94FB1FE88113
:10400800F98131961EB5119310E01EBD0DB511272B
:1040180007FD1FEF112311F40C940A20E881F981A0
:104028001EB51193FE01A081B1811196A083B183C1
:104038000C94E51F289A15E00E94EB330895289800
:1040480012E01EBD0DB5112707FD1FEF112311F456
:104058000C9426201A811EBD0DB5112707FD1FEFF0
:10406800112311F40C943020088119811EBD0DB55F
:10407800112707FD1FEF112311F40C943B20088131
:104088001981102F1EBD0DB5112707FD1FEF112334
:1040980011F40C944720289A16E00E94EB330895F7
:1040A800299818811EBD0DB5112707FD1FEF112393
:1040B80011F40C94572011E00E94EB33299A0895CB
:1040C80021971A8124E00E9436371F9319811F70A7
:1040D8000F91100F1883CF93DF9312E01A93198171
:1040E800012F11271A930A930E942320DF91CF9161
:1040F80008952297FE013196EF93FF931B81FF915C
:10410800EF911193FE01EF93FF931A81FF91EF91C5
:104118001193CF93DF931BE01A9309811A811A93A5
:104128000A930E942320DF91CF9108952197219A25
:10413800209A229A259A279A2F9811E51CBDADE45A
:10414800B0E010E00E948D381DB5188308952297BD
:10415800FE01FA93EA9310E001E000831183EF93E4
:10416800FF930C811D81FF91EF911A930A93A0810F
:10417800B18128813981B31709F4A21710E011F031
:1041880008F01FEF112311F00C94DF20CF93DF9379
:1041980010E01A930E945420DF91CF91EA81FB81AD
:1041A800A081B1811196A083B183BB2311F4AA2306
:1041B80011F00C94BD20249608952A9810E004E18B
:1041C8000E94DC33289A299A2A9A10E00AE00E9471
:1041D800DC33CF93DF931BE01A931FEF0FEF1A9393
:1041E8000A930E942320DF91CF91CF93DF9313E0AE
:1041F8001A9318E900E01A930A930E942320DF918A
:10420800CF9110E001E00E94DC3311274A991FEF9B
:10421800112311F40C940921CF93DF9315E01A931D
:1042280010E00AE01A930A930E942320DF91CF91AD
:1042380010E004E60E94DC33CF93DF931EEF1A935D
:104248001EEF1A930E947D20DF91CF91CF93DF93C9
:1042580015E01A931FE100E41A930A930E942320A1
:10426800DF91CF910895229710E008EC0E94DC338B
:10427800CF93DF9310E01A9318E004EA1A930A9395
:104288000E942320DF91CF9112E00E94EB33CF935D
:10429800DF9313E01A9318E900E01A930A930E9437
:1042A8002320DF91CF912998CF93DF9313E51A93B9
:1042B8000E94C51FDF91CF91FE01FA93EA9310E0A7
:1042C80001E00083118314E000E01A930A93A081AF
:1042D800B18128813981B31709F4A21710E011F0D0
:1042E80008F01FEF112311F00C94962111274A9919
:1042F8001FEF112311F40C947A21CF93DF9310E070
:104308001A930E94C51FDF91CF91EA81FB81A0819A
:10431800B1811196A083B183BB2311F4AA2311F0B4
:104328000C946D2124960E94BC1F299A089510E0D0
:1043380003E00E94DC33CF93DF930E943721DF91A3
:10434800CF9110E003E00E94DC33CF93DF9310E0BD
:1043580000E21A930A930E94AB20DF91CF9108954F
:104368002998CF93DF9313E51A930E94C51FDF9115
:10437800CF91CF93DF931FEE1A930E94C51FDF9151
:10438800CF91CF93DF931EE61A930E94C51FDF914A
:10439800CF91CF93DF9314E41A930E94C51FDF9146
:1043A800CF91CF93DF9310E01A930E94C51FDF913E
:1043B800CF91CF93DF9310E01A930E94C51FDF912E
:1043C800CF91CF93DF9310E01A930E94C51FDF911E
:1043D800CF91CF93DF9310E01A930E94C51FDF910E
:1043E800CF910E94BC1F299A08952998CF93DF93F3
:1043F80013E51A930E94C51FDF91CF91CF93DF93E6
:104408001FEE1A930E94C51FDF91CF91CF93DF93C0
:104418001EE61A930E94C51FDF91CF91CF93DF93B9
:1044280014E41A930E94C51FDF91CF91CF93DF93B5
:1044380010E01A930E94C51FDF91CF91CF93DF93AD
:1044480010E01A930E94C51FDF91CF91CF93DF939D
:1044580010E01A930E94C51FDF91CF91CF93DF938D
:1044680010E01A930E94C51FDF91CF910E94BC1FD4
:10447800299A08952998CF93DF9315E41A930E94F7
:10448800C51FDF91CF91CF93DF9318E71A930E944E
:10449800C51FDF91CF91CF93DF9319E61A930E943E
:1044A800C51FDF91CF91CF93DF9314E71A930E9432
:1044B800C51FDF91CF91CF93DF9310E01A930E942D
:1044C800C51FDF91CF91CF93DF9310E01A930E941D
:1044D800C51FDF91CF91CF93DF9310E01A930E940D
:1044E800C51FDF91CF91CF93DF9310E01A930E94FD
:1044F800C51FDF91CF910E94BC1F299A08950E9481
:10450800F92113E008EE0E94DC330E943E2211E0FC
:1045180004EF0E94DC3308952197FE01FA93EA9391
:1045280010E0108312E01A931081088101171FEF21
:1045380008F01127112311F00C94BD22CF93DF93BB
:104548001EE31A930E94B421DF91CF9110E004E694
:104558000E94DC330E943E2210E004E60E94DC3315
:10456800E981FA81108113951083112311F00C94BD
:104578009922239608952197FE01FA93EA9310E36E
:10458800108316E71A931081088101171FEF08F0AE
:104598001127112311F00C94E8220E943E22CF9398
:1045A800DF931B811A930E94B421DF91CF9110E011
:1045B80009E10E94DC33E981FA81108113951083A7
:1045C800112311F00C94C82223960E943E220895CC
:1045D80021971981112311F40C94032311270091B9
:1045E8003B0674E0071B60E010F4062F03C00617B3
:1045F800E0F31FEF00933B0618830C941323112755
:1046080000913B0674E0070F6FEF10F4062F04C00B
:10461800061709F0D8F71FEF00933B06188310918F
:104628003B06E0E0F0E00E94143431961881112333
:1046380011F40C9441231091D205103010E009F4C4
:104648001FEF112311F40C941F2311E0F894109319
:10465800D20547FC7894CF93DF9310913B061A93C9
:1046680010913B061A930E947D20DF91CF9110E0B4
:10467800F8941093D20547FC789408952197FE0189
:10468800FA93EA9310E0108311E11A9310810881DC
:1046980001171FEF08F01127112311F00C9495232F
:1046A800FE013496EF93FF93EEE3F6E0EF93FF936A
:1046B8001B81012F1127A8E0B0E0E89445F80E947B
:1046C8006537FF91EF91E00FF11FBF91AF91E8942B
:1046D80044F80E94D13610E009F41FEF112311F4B9
:1046E8000C948C23EEE3F6E0EF93FF931B81012FEC
:1046F8001127A8E0B0E0E89445F80E946537FF91DB
:10470800EF91E00FF11F3796119123960C949723A0
:10471800E981FA81108113951083112311F00C940B
:104728004B23239610E0089522970E94CA31113630
:1047380018F01B3708F410521883CF93DF9318E052
:10474800412A0EEE11E31A930A93FE013296108164
:104758000E94F736DF91CF911881193310E011F0DC
:1047680008F01FEF112311F40C94C223188117537A
:1047780000E10E944C3719830C94C8231881105308
:1047880000E10E944C3719830E94CA31113618F093
:104798001B3708F410521883CF93DF9318E0412A8F
:1047A8000EEE11E31A930A93FE01329610810E94CD
:1047B800F736DF91CF911881193310E011F008F026
:1047C8001FEF112311F40C94F22319811F93188100
:1047D8000F91100F175319830C94F92319811F9304
:1047E80018810F91100F105319831981089521977B
:1047F8000E94CA31113618F01B3708F4105218837A
:10480800CF93DF9318E0412A0EEE11E31A930A932F
:10481800FE01329610810E94F736DF91CF91188100
:10482800193510E009F41FEF112311F40C94212419
:104838001FEF0C9424240C94242410E00C942424BA
:104848000895CF93DF9318E0412A0EEE11E31A93EF
:104858000A93EFE3F2E7B591BB2311F00E94A83564
:10486800E0E8F5E00E94AE351DE00E94F7361AE058
:104878000E94F736DF91CF9108952797CF93DF9362
:1048880018E0412A0EEE11E31A930A931DE00E94E4
:10489800F7361AE00E94F736DF91CF91CF93DF9376
:1048A80027974F92FE01EF93FF933196FA93EA937D
:1048B80016E01A9317EF41221FEB4122E3EDF5E0D2
:1048C8000E94AE3516E01F9318810F91011B102F1F
:1048D800FF91EF91108323964F900E944223DF911E
:1048E800CF911A831A811A3111F00C94D224E3ED76
:1048F800F5E037961FEB4122E89441F800E00E946A
:10490800D3341C830B83CF93DF930B811C811A93C1
:104918000A930E946A1EDF91CF91112311F40C941F
:10492800B924CF93DF9318E0412A0EEE11E31A93CE
:104938000A93E6E4F2E7B591BB2311F00E94A8358B
:10494800E8E2F6E00E94AE35EFE4F2E7B591BB236A
:1049580011F00E94A8351DE00E94F7361AE00E9467
:10496800F736DF91CF910C94D024CF93DF9318E0E2
:10497800412A0EEE11E31A930A93E7E5F2E7B5919F
:10498800BB2311F00E94A8351DE00E94F7361AE0FB
:104998000E94F736DF91CF910C94BA29193111F0A2
:1049A8000C94C325CF93DF9366974F92FE01EF9344
:1049B800FF933196FA93EA9315E11A9317EF412280
:1049C8001FEB41221CE50E94F73615E11F93188161
:1049D8000F91011B102FFF91EF91108323964F9099
:1049E8002D974F92FE01EF93FF933196FA93EA9336
:1049F8001CE01A9317EF41221FEB4122E3EDF5E08B
:104A080037960E94AE35EAE3F2E7B591BB2311F081
:104A18000E94A8351CE01F9318810F91011B102FCD
:104A2800FF91EF91108323964F9017E21A93E0E8D5
:104A3800F5E0FA93EA930E949716DF91CF9111233C
:104A480011F40C94AA25E8E2F6E0EF93FF9331966F
:104A5800FA93EA931CE01A9317EF41221FEB4122C5
:104A6800E0E8F5E00E94AE351CE01F9318810F9135
:104A7800011B102FFF91EF9110832396CF93DF93A3
:104A880066974F92FE01EF93FF933196FA93EA935C
:104A980015E11A9317EF41221FEB41221CE50E94F2
:104AA800F73615E11F9318810F91011B102FFF9105
:104AB800EF91108323964F902D974F92FE01EF931D
:104AC800FF933196FA93EA931CE01A9317EF412269
:104AD8001FEB4122E0E8F5E00E94AE351CE01F9391
:104AE80018810F91011B102FFF91EF9110832396CE
:104AF8004F90E8E2F6E03D96FA93EA930E94F715A4
:104B0800DF91CF91CF93DF9318E0412A0EEE11E3A6
:104B18001A930A93E6E4F2E7B591BB2311F00E94D9
:104B2800A835E8E2F6E00E94AE35EFE4F2E7B59189
:104B3800BB2311F00E94A8351DE00E94F7361AE049
:104B48000E94F736DF91CF910C94C125CF93DF9364
:104B580018E0412A0EEE11E31A930A93E7E5F2E70B
:104B6800B591BB2311F00E94A8351DE00E94F736CD
:104B78001AE00E94F736DF91CF910C94BA291231CE
:104B880011F00C940E26E3EDF5E037961FEB412269
:104B9800E89441F800E00E94D3341C830B83CF9340
:104BA800DF930B811C811A930A930E946A1EDF917E
:104BB800CF91112311F40C94EC2511E0712FA3E08F
:104BC800B6E048E256E000E20E94D0380C940C2689
:104BD800CF93DF9318E0412A0EEE11E31A930A935C
:104BE800E7E5F2E7B591BB2311F00E94A8351DE077
:104BF8000E94F7361AE00E94F736DF91CF9113E052
:104C0800712FA3E0B6E048E256E000E20E94D038F7
:104C18000C94BA29113111F00C94EF26CF93DF933D
:104C280066974F92FE01EF93FF933196FA93EA93BA
:104C380015E11A9317EF41221FEB41221CE50E9450
:104C4800F73615E11F9318810F91011B102FFF9163
:104C5800EF91108323964F902D974F92FE01EF937B
:104C6800FF933196FA93EA931CE01A9317EF4122C7
:104C78001FEB4122E3EDF5E037960E94AE35EAE3FB
:104C8800F2E7B591BB2311F00E94A8351CE01F93F1
:104C980018810F91011B102FFF91EF91108323961C
:104CA8004F9017E21A93E0E8F5E0FA93EA930E942E
:104CB8009716DF91CF91112311F40C94CD26E8E2D9
:104CC800F6E0EF93FF933196FA93EA931CE01A9378
:104CD80017EF41221FEB4122E0E8F5E00E94AE35D4
:104CE8001CE01F9318810F91011B102FFF91EF916A
:104CF80010832396CF93DF9366974F92FE01EF932D
:104D0800FF933196FA93EA9315E11A9317EF41222C
:104D18001FEB41221CE50E94F73615E11F9318810D
:104D28000F91011B102FFF91EF91108323964F9045
:104D38002D974F92FE01EF93FF933196FA93EA93E2
:104D48001CE01A9317EF41221FEB4122E0E8F5E03F
:104D58000E94AE351CE01F9318810F91011B102F84
:104D6800FF91EF91108323964F90E8E2F6E03D968D
:104D7800FA93EA930E94F715DF91CF9111E0712F12
:104D8800A3E0B6E048E256E000E20E94D0380C9476
:104D9800ED26CF93DF9318E0412A0EEE11E31A9324
:104DA8000A93E7E5F2E7B591BB2311F00E94A83515
:104DB8001DE00E94F7361AE00E94F736DF91CF9186
:104DC80013E0712FA3E0B6E048E256E000E20E944B
:104DD800D0380C94BA29133111F00C94FE2612E045
:104DE800712FA3E0B6E048E256E000E20E94D03816
:104DF8000C94BA29143111F00C946127CF93DF93E6
:104E080018E0412A0EEE11E31A930A93EFE3F2E752
:104E1800B591BB2311F00E94A835E8E2F6E00E94A4
:104E2800AE35E7E3F2E7B591BB2311F00E94A83550
:104E38000091CD051091CE052091CF053091D00578
:104E48000F931F932F933F9310E01F9310E01F932E
:104E580010E21F93E89445F80E940036E7E3F2E772
:104E6800B591BB2311F00E94A835E8E2F6E03D9623
:104E780001911191219131910F931F932F933F939A
:104E880010E01F9310E01F9310E21F93E89445F879
:104E98000E9400361DE00E94F7361AE00E94F7369D
:104EA800DF91CF9114E0712FA3E0B6E048E256E01D
:104EB80000E20E94D0380C94BA29153111F00C94F4
:104EC8008727CF93DF9318E0412A0EEE11E31A9358
:104ED8000A93E8E6F2E7B591BB2311F00E94A835E2
:104EE8001DE00E94F7361AE00E94F736DF91CF9155
:104EF80013E0712FA3E0B6E048E256E000E20E941A
:104F0800D0380C94BA29103811F00C949327CF9309
:104F1800DF930E949022DF91CF910C94BA2910322E
:104F280011F00C940F28CF93DF9366974F92FE01F0
:104F3800EF93FF933196FA93EA9315E11A9317EFDB
:104F480041221FEB41221CE50E94F73615E11F9311
:104F580018810F91011B102FFF91EF911083239659
:104F68004F902D974F92FE01EF93FF933196FA934E
:104F7800EA931CE01A9317EF41221FEB4122E8E75E
:104F8800F2E7B591BB2311F00E94A8351CE01F93EE
:104F980018810F91011B102FFF91EF911083239619
:104FA8004F901FE31A93E0E8F5E0FA93EA930E9422
:104FB8009716DF91CF91112311F40C940D28CF93FC
:104FC800DF9318E0412A0EEE11E31A930A93ECE7F7
:104FD800F2E7B591BB2311F00E94A835E0E8F5E0AF
:104FE8000E94AE351DE00E94F7361AE00E94F7369F
:104FF800DF91CF91CF93DF93E0E8F5E0FA93EA935E
:105008000E943418DF91CF911095112311F40C945C
:10501800E3270C94BA29113211F00C946928CF9324
:10502800DF9318E0412A0EEE11E31A930A93E2E89F
:10503800F2E7B591BB2311F00E94A835E8E2F6E04B
:105048000E94AE35E7E3F2E7B591BB2311F00E9469
:10505800A8350091CD051091CE052091CF0530914E
:10506800D0050F931F932F933F9310E01F9310E0E9
:105078001F9310E21F93E89445F80E940036E7E377
:10508800F2E7B591BB2311F00E94A835E8E2F6E0FB
:105098003D9601911191219131910F931F932F9377
:1050A8003F9310E01F9310E01F9310E21F93E894C2
:1050B80045F80E9400361DE00E94F7361AE00E946B
:1050C800F736DF91CF910C94BA29163111F00C9470
:1050D8009328CF93DF931FEF1A930E94EC22DF915E
:1050E800CF91CF93DF9318E0412A0EEE11E31A9384
:1050F8000A93E9E8F2E7B591BB2311F00E94A835BD
:1051080010913B06412F0E94EA361DE00E94F736B7
:105118001AE00E94F736DF91CF910C94BA29173123
:1051280011F00C94BD28CF93DF9310E01A930E94DE
:10513800EC22DF91CF91CF93DF9318E0412A0EEE56
:1051480011E31A930A93E9E8F2E7B591BB2311F04A
:105158000E94A83510913B06412F0E94EA361DE0B7
:105168000E94F7361AE00E94F736DF91CF910C942F
:10517800BA29183111F00C941529E3EDF5E03796AA
:105188001FEB4122E89441F80FEF0E94D334102F0F
:1051980010933B0610913B06E0E0F0E00E941434C7
:1051A80031961091D205103010E009F41FEF112349
:1051B80011F40C94D52811E0F8941093D20547FC0B
:1051C8007894CF93DF9310913B061A9310913B0686
:1051D8001A930E947D20DF91CF9110E0F8941093EC
:1051E800D20547FC7894CF93DF9318E0412A0EEE5E
:1051F80011E31A930A93E9E8F2E7B591BB2311F09A
:105208000E94A83510913B06412F0E94EA361DE006
:105218000E94F7361AE00E94F736DF91CF910C947E
:10522800BA29103A11F00C944629CF93DF9318E06D
:10523800412A0EEE11E31A930A93E6E9F2E7B591D3
:10524800BB2311F00E94A835EEECF6E0EF93FF9334
:105258001091CB05012F1127ABE0B0E0E89445F899
:105268000E946537FF91EF91E00FF11F0E94AE3564
:105278001DE00E94F7361AE00E94F736DF91CF91C1
:105288000C94BA29123A11F00C94A329CF93DF9306
:1052980018E0412A0EEE11E31A930A93EFE9F2E7B8
:1052A800B591BB2311F00E94A8351DE00E94F73686
:1052B8001AE00E94F736DF91CF91CF93DF930E94D7
:1052C800FB23DF91CF91112311F40C948A29CF93FA
:1052D800DF9318E0412A0EEE11E31A930A93E4ECE7
:1052E800F2E7B591BB2311F00E94A8351DE00E949A
:1052F800F7361AE00E94F736DF91CF9112E00CEBF7
:105308000E94DC330E942F7E0C94A129CF93DF9357
:1053180018E0412A0EEE11E31A930A93E3EDF2E73F
:10532800B591BB2311F00E94A8351DE00E94F73605
:105338001AE00E94F736DF91CF910C94BA29CF93E7
:10534800DF9318E0412A0EEE11E31A930A93E4EE74
:10535800F2E7B591BB2311F00E94A8351DE00E9429
:10536800F7361AE00E94F736DF91CF9108950E9430
:105378004C1E0E94661E0E94561E10E8412A789410
:105388000E94BF310E94CC3810E00AE00E94DC3352
:10539800CF93DF9318E0412A0EEE11E31A930A9394
:1053A800EBEFF2E7B591BB2311F00E94A8351DE0A1
:1053B8000E94F7361AE00E94F736DF91CF9110E08D
:1053C8001093CB0510E01093CC0510E01093D10595
:1053D80010910306103010E011F008F01FEF1F9332
:1053E8001091CB051B3010E009F01FEF0F9110232F
:1053F800112311F40C943D2AA3E0B6E048E256E0EC
:1054080070E00E94E7381093660710916607113024
:1054180011F00C94142A14E01093CB050C943D2A37
:10542800123011F00C941D2A16E01093CB050C9441
:105438003D2A133011F00C94302ACF93DF93EEE716
:10544800F5E0FA93EA930E942C1ADF91CF9118E0C5
:105458001093CB050C943D2A143011F00C943D2A7E
:10546800459810E010933D0615E01093CB050C9479
:105478003D2A1091CC05103011F00C94522A1127B6
:1054880036991FEF112311F40C94502A11E0109350
:10549800CC0519E01093CB050C946E2A113011F04D
:1054A8000C946E2A112736991FEF1095112311F4C9
:1054B8000C946C2A10E01093CC05459A10E01093D8
:1054C8003D0610E008EC0E94DC3311E01093CB0598
:1054D8000C946E2A1091CB05103011F00C94D12A3F
:1054E800CF93DF930E949A20DF91CF91CF93DF93E0
:1054F80018E0412A0EEE11E31A930A93E0E1F3E76C
:10550800B591BB2311F00E94A8351DE00E94F73623
:105518001AE00E94F736DF91CF910E94E120CF93E5
:10552800DF9318E0412A0EEE11E31A930A93EDE196
:10553800F3E7B591BB2311F00E94A8351DE00E9446
:10554800F7361AE00E94F736DF91CF91CF93DF93B9
:105558000E943721DF91CF91CF93DF931FE01A93F9
:1055680014E01A930E946420DF91CF91CF93DF93C8
:1055780010913B061A9310913B061A930E947D20C6
:10558800DF91CF9110E0F8941093D20547FC7894FE
:1055980011E01093CB050C94AF2D113011F00C9441
:1055A800222CCF93DF9318E0412A0EEE11E31A93D1
:1055B8000A93EAE2F3E7B591BB2311F00E94A835FC
:1055C8001DE00E94F7361AE00E94F736DF91CF916E
:1055D800CF93DF930E94901FDF91CF91112311F495
:1055E8000C94FF2BCF93DF9310E001E01A930A93FA
:1055F8000E946A1EDF91CF91112311F40C941D2B88
:10560800CF93DF9318E0412A0EEE11E31A930A9321
:10561800E7E3F3E7B591BB2311F00E94A8351DE03D
:105628000E94F7361AE00E94F736DF91CF910C946A
:10563800F82BCF93DF9366974F92FE01EF93FF937A
:105648003196FA93EA9315E11A9317EF41221FEB6B
:1056580041221CE50E94F73615E11F9318810F912E
:10566800011B102FFF91EF91108323964F902D97D8
:105678004F92FE01EF93FF933196FA93EA931CE061
:105688001A9317EF41221FEB4122E3E4F3E7B591A8
:10569800BB2311F00E94A8351CE01F9318810F91BD
:1056A800011B102FFF91EF91108323964F9017E263
:1056B8001A93E0E8F5E0FA93EA930E949716DF91CF
:1056C800CF91112311F40C94E12BE8E2F6E0EF936B
:1056D800FF933196FA93EA931CE01A9317EF41224D
:1056E8001FEB4122E0E8F5E00E94AE351CE01F9375
:1056F80018810F91011B102FFF91EF9110832396B2
:10570800CF93DF9366974F92FE01EF93FF93319605
:10571800FA93EA9315E11A9317EF41221FEB4122FE
:105728001CE50E94F73615E11F9318810F91011BA4
:10573800102FFF91EF91108323964F902D974F9242
:10574800FE01EF93FF933196FA93EA931CE01A93C4
:1057580017EF41221FEB4122E0E8F5E00E94AE3549
:105768001CE01F9318810F91011B102FFF91EF91DF
:10577800108323964F90E8E2F6E03D96FA93EA9379
:105788000E94F715DF91CF91CF93DF9318E0412A5C
:105798000EEE11E31A930A93E7E3F3E7B591BB23FF
:1057A80011F00E94A8351DE00E94F7361AE00E9409
:1057B800F736DF91CF910C94F82BCF93DF9318E055
:1057C800412A0EEE11E31A930A93E9E4F3E7B5913F
:1057D800BB2311F00E94A8351DE00E94F7361AE09D
:1057E8000E94F736DF91CF910E94681E13E0109354
:1057F800CB050C94202CCF93DF9318E0412A0EEEB2
:1058080011E31A930A93E5E6F3E7B591BB2311F088
:105818000E94A8351DE00E94F7361AE00E94F7366C
:10582800DF91CF9114E110933D0610913D0610933E
:105838003C061BE01093CB050C94AF2D133011F0F0
:105848000C94282C0C94AF2D143011F00C94AA2C25
:1058580045980E94661E10E010933D06CF93DF9393
:10586800EEE7F5E0FA93EA9366974F92FE01EF931D
:10587800FF933196FA93EA9315E11A9317EF4122B1
:105888001FEB41221CE50E94F73615E11F93188192
:105898000F91011B102FFF91EF91108323964F90CA
:1058A8002D974F92FE01EF93FF933196FA93EA9367
:1058B8001CE01A9317EF41221FEB4122E0E8F5E0C4
:1058C8000E94AE351CE01F9318810F91011B102F09
:1058D800FF91EF91108323964F9010E001E0009321
:1058E800D8011093D9010E944A15DF91CF911093E6
:1058F8006107CF93DF9300917E0510917F051A937E
:105908000A930E94A519DF91CF91109361070E9415
:10591800252400E010E020E030E00093CD0510934E
:10592800CE052093CF053093D005CF93DF930E9407
:105938003721DF91CF9110E0F8941093D20547FCFE
:10594800789415E01093CB050C94AF2D153011F019
:105958000C94452DCF93DF9300917E0510917F0520
:105968001A930A93E0E4F7E08F011A930A9310E080
:1059780000E21A930A93EEE3F7E0FA93EA930E949F
:105988000B1BDF91CF911093610711274A991FEFE5
:10599800112311F40C94C92C2998E2E6F7E0FA9344
:1059A800EA9310E000E00083118310E00FE11A93FE
:1059B8000A93A081B18128813981E0E8BE273E277A
:1059C800B31709F4A21710E011F008F01FEF112324
:1059D80011F00C94242DE0E4F7E000916207109197
:1059E8006307E00FF11F11911EBD11E00E94EB3318
:1059F8000DB5112707FD1FEF112311F40C94FC2C92
:105A0800A091CD05B091CE05E091CF05F091D005DC
:105A1800119608F43196A093CD05B093CE05E09386
:105A2800CF05F093D005EA81FB81A081B181119661
:105A3800A083B183B03811F4A03011F00C94DF2C9E
:105A48002496299ACF93DF9300917E0510917F05C4
:105A58001A930A930E94BD1ADF91CF91112311F472
:105A68000C94432DCF93DF93EEE7F5E0FA93EA9396
:105A78000E942C1ADF91CF9118E01093CB050C945B
:105A8800AF2D163011F00C946D2D459A12E310933A
:105A98003D0610913D0610933C06CF93DF9318E026
:105AA800412A0EEE11E31A930A93E8E8F3E7B59159
:105AB800BB2311F00E94A8351DE00E94F7361AE0BA
:105AC8000E94F736DF91CF9117E01093CB050C9425
:105AD800AF2D173011F00C94732D0C94AF2D183096
:105AE80011F00C94822D459A10E010933D060E9407
:105AF800681E13E01093CB050C94AF2D193011F0EC
:105B08000C94A92DCF93DF9318E0412A0EEE11E3F0
:105B18001A930A93E7E9F3E7B591BB2311F00E94C2
:105B2800A8351DE00E94F7361AE00E94F736DF918B
:105B3800CF911EE110933D0610913D0610933C064F
:105B48001BE01093CB050C94AF2D1B3011F00C9477
:105B5800AF2D0C94AF2D0E948731112311F40C94B2
:105B6800112E0E94B7310093C9051093CA050E94EF
:105B7800923110936407112730991FEF103010E00D
:105B880009F41FEF112311F40C94CF2D1091640721
:105B9800105F10936407EEE3F5E0EF93FF93109125
:105BA8006407012F1127000F111FFF91EF91E00FDC
:105BB800F11F019111910093670710936807CF9324
:105BC800DF9300916707109168071A930A930E9460
:105BD8006A1EDF91CF91112311F40C94FC2D11E072
:105BE800712FA3E0B6E048E256E000E20E94D03808
:105BF8000E94B7310F931F9310E000E098011F91A6
:105C08000F91131709F4021710E009F41FEF11237D
:105C180011F40C94FC2D0E94BF3112E00E94B73899
:105C2800112311F40C943C2ECF93DF931FEF1A939A
:105C38000E94EC22DF91CF91CF93DF9318E0412AA5
:105C48000EEE11E31A930A93E9E8F2E7B591BB2344
:105C580011F00E94A83510913B06412F0E94EA36A8
:105C68001DE00E94F7361AE00E94F736DF91CF91C7
:105C780013E00E94B738112311F40C94672ECF93C8
:105C8800DF9310E01A930E94EC22DF91CF91CF931B
:105C9800DF9318E0412A0EEE11E31A930A93E9E81C
:105CA800F2E7B591BB2311F00E94A83510913B068D
:105CB800412F0E94EA361DE00E94F7361AE00E9442
:105CC800F736DF91CF9111E00E94B738112311F414
:105CD8000C94932E6FE077E221E030E0E9E3F6E000
:105CE8000E94F433112311F40C94932ECF93DF9375
:105CF8000091390610913A061A930A930E946A1E77
:105D0800DF91CF91112311F40C94932E11E0712F90
:105D1800A3E0B6E048E256E000E20E94D03810E086
:105D28000E94B738112311F40C94A32E11E0712F9F
:105D3800A3E0B6E048E256E000E20E94D0380E94B4
:105D4800E731112311F40C94AC2F0E94CA3111369B
:105D580018F01B3708F4105210936507CF93DF93A0
:105D680018E0412A0EEE11E31A930A931091650781
:105D78000E94F736DF91CF911091D105103011F0C4
:105D88000C94F22E10916507103211F00C94CE2E5F
:105D98000C94D22E1D3011F00C94D72E10E01093D5
:105DA800D1050C94F02E11E010936407E3EDF5E0B3
:105DB800EF93FF9310916407012F11273F912F91C3
:105DC800020F131F0F931F9310916507FF91EF9117
:105DD800119311E01093D1050C94AC2F113011F0F0
:105DE8000C94602F109165071D3011F00C94192F39
:105DF800E3EDF5E0EF93FF9310E0012F11273F91BA
:105E08002F91020F131F0F931F9310916407FF9197
:105E1800EF911193CF93DF930E944124DF91CF91AB
:105E280010E01093D1050C945E2F103211F00C94F1
:105E3800372FE3EDF5E0EF93FF9310E0012F1127E3
:105E48003F912F91020F131F0F931F931091640717
:105E5800FF91EF91119310E01093640712E01093F3
:105E6800D1050C945E2F11270091640776E007177F
:105E780020F40395009364071FEF1095112311F484
:105E88000C944B2F10E01093D1050C945E2FE3ED8A
:105E9800F5E0EF93FF9310916407012F11273F91CD
:105EA8002F91020F131F0F931F9310916507FF91F6
:105EB800EF9111930C94AC2F123011F00C94AC2F7D
:105EC800109165071D3011F00C94852FE3EDF5E076
:105ED800EF93FF9310E0012F11273F912F91020FAD
:105EE800131FF8013796109164071193CF93DF932E
:105EF8000E944124DF91CF9110E01093D1050C94BA
:105F0800AA2F11270091640778E2071720F4039558
:105F1800009364071FEF1095112311F40C94992F27
:105F280010E01093D1050C94AA2FE3EDF5E0EF9360
:105F3800FF9310916407012F11273F912F91020FB2
:105F4800131FF80137961091650711930C94AC2F25
:105F580010913D06103010E011F008F01FEF1123EA
:105F680011F40C94C72F1FEF00913C06002309F091
:105F78001095112311F40C94C72F00E206B9109163
:105F88003D0610933C060C94EC290000FECFF894D3
:105F980018E008E61EBF0DBF1127E0E1F0E0A0E021
:105FA800B0E03196319711F01D93FCCFA0E0B1E03D
:105FB800E0E0F0E13196319711F01D93FCCFC8E68F
:105FC800D9E0F8941FE7412212E01093D701AEE31D
:105FD800B5E0EBEAF3E720E430E019D016E01093DF
:105FE80007061093050618E010930606109304069A
:105FF800AEE3B6E0E9E5F4E720E930E008D0AEEC3E
:10600800B6E0EBEEF3E72EE630E001D007C0215012
:10601800304018F015911D93FACF089516E11093AA
:10602800080116BD14E015BD11E010936E0018E1CB
:106038001093C10016E21093C40010E01093C5003D
:1060480010E0109370011093710110937201109178
:10605800C10010681093C10010E01093090110935B
:106068000A0110930B0116E01093C2001091C600AC
:106078002C9A2E9A279A259A249A0000000000004C
:106088001CE51CBD0000000000000000000000002E
:10609800000000000DB50EB51127109302011093F2
:1060A800010110930401109303011093060110934A
:1060B800050111B1107F11B912B1107F12B911B1D8
:1060C8001F7011B9442455240C94BB29EF93FF93F6
:1060D8000F931F931FB71F931091080106B5100F58
:1060E80016BD1FE7412210913C06112319F01150EB
:1060F80010933C061091D7011A951093D70109F017
:1061080080C012E01093D70110910001112309F00B
:106118005BC04F93112700271098089A40E00E940F
:106128006F31109A08981198099A41E00E946F31CE
:10613800119A099812980A9A42E00E946F31129AAD
:106148000A9813980B9A43E00E946F31139A0B98A0
:106158004F91E8940F93012FF09102011F27F091BE
:106168000401EF2FE12310951023E12BE0930401A4
:10617800FE27FE2309F06894E0910601EF2BE093D7
:106188000601009302011F91012FF09101011F27C1
:10619800F0910301EF2FE12310951023E12BE093F9
:1061A8000301FE27FE2309F06894E0910501EF2B17
:1061B800E0930501009301013EF4F0910701FF3FD0
:1061C80019F0F395F0930701112709B104FB10F9B1
:1061D80009B105FB11F909B106FB12F909B107FB71
:1061E80013F90FEF1027012F1725782C812210950E
:1061F8001023812A10E07094712618251721912AFE
:10620800702E10E8412A1F911FBF1F910F91FF9117
:10621800EF911895EF93FF930F931F931FB71F9359
:1062280010910B01112331F41091C1001F7D1093BF
:10623800C1001BC000910A011127ECE0F1E0E00F5A
:10624800F11F10811093C60010910B011A9510933D
:106258000B0129F41091C1001F7D1093C100039513
:10626800043609F4002700930A011F911FBF1F91EC
:106278000F91FF91EF911895EF93FF930F931F9351
:106288001FB71F9310917201143619F40091C600BC
:106298001BC01091C6001F93112700917001E3E7FE
:1062A800F1E0E00FF11F1F91108310917201139517
:1062B800109372010395043609F4002700937001C6
:1062C8000091C00007FDDECF1F911FBF1F910F91E6
:1062D800FF91EF91189500000000000008940499C0
:1062E8008894001F111F089405998894001F111F96
:1062F800089406998894001F111F08940799889498
:10630800001F111F089510910501112329F4109100
:106318000601112309F408951FEF08950E94A4317E
:106328001123E1F310E0312F0E94AF31112331F432
:106338003395132F1F7091F3132FF6CF132F089552
:1063480010910301112329F410910401112309F478
:1063580008951FEF0895F894A3E0B1E00E949838DB
:1063680047FC78940895F894009103011091040172
:1063780047FC78940895F894112710930601109318
:1063880005011093070147FC789408951091720154
:106398001123E1F3009171011127E3E7F1E0E00F28
:1063A800F11F1081F894E0917201EA95E09372016F
:1063B80047FC7894009171010395043609F400278D
:1063C800009371010895112700917201002309F0CB
:1063D8001095089500910B010436E1F3F8940091AB
:1063E8000901ECE0F1E0E00F0027F01F10830091B5
:1063F8000B01039500930B010091090103950436E5
:1064080009F40027009309010091C100006200937C
:10641800C10047FC7894089510E01093FF041FEF23
:106428001093AC041093AD041093AE041093AF0412
:106438000DC05CC00F931EBD00000DB506FDFBCF5F
:106448000DB507FFFDCF1EB50F9108950CB50F933D
:106458000EE50CBD2C9A0DE01FEFECDF0A95E1F775
:106468002C9810E4E7DF10E0E5DF10E0E3DF10E050
:10647800E1DF10E0DFDF15E9DDDF0DE01FEFDADF38
:10648800113011F00A95D1F72C9A1FEFD3DF0023B2
:1064980021F40F910CBD10E00895A4E677270AE0D7
:1064A80011270E94DC332C9811E4C4DF10E0C2DF0E
:1064B80010E0C0DF10E0BEDF10E0BCDF1FEFBADF86
:1064C800B0E11FEFB7DF103011F0BA95D1F7712F97
:1064D8002C9A1FEFAFDFAA9511F0772301F7112748
:1064E800772309F41FEF0F910CBD08952C981FEF27
:1064F800A1DF1AE49FDF10E09DDF10E09BDF10E0D2
:1065080099DF10E097DF1FEF00E21FEF93DF1030F5
:1065180029F00A95D1F72C9A112708950AEF1FEF51
:1065280089DF1E3F29F00A95D1F72C9A1127089583
:1065380000E1EBEDF3E01FEF7DDF11930A95D9F74A
:106548001FEF78DF1FEF76DF2C9A1FEF73DF1FEF47
:1065580008952C981FEF6EDF11E56CDF1D816ADF4F
:106568001C8168DF1B8166DF1A8164DF00E21FEF90
:1065780061DF103029F00A95D1F72C9A1127089578
:10658800A8EEB3E01FEF56DF1E3F29F01197D1F7B1
:106598002C9A11270895A0E0B2E0E881F9811FEF55
:1065A80049DF11931197D9F71FEF44DF1FEF42DF3F
:1065B8002C9A1FEF3FDF1FEF08952C981FEF3ADF4B
:1065C80018E538DF1D8136DF1C8134DF1B8132DF9F
:1065D8001A8130DF00E21FEF2DDF103029F00A9515
:1065E800D1F72C9A112708951FEF24DF1FEF22DF20
:1065F8001EEF20DFA0E0B2E0E881F98111911ADFF7
:106608001197E1F71FEF16DF1FEF14DF7FEF1FEF82
:1066180011DF712F1FEF0EDF1F3FE1F72C9A1FEFDD
:1066280009DF1FEF08950A811B812C813D81ECEA67
:10663800F4E06081061759F46181161741F462810C
:10664800261729F46381361711F41FEF0895019373
:106658001193219331936091FF047727060F171F39
:10666800271F371F000F111F221F331F7A830B8329
:106678001C832D8300E00F936CDF0F91112379F4B5
:106688000A95C9F7112359F40FEFECEAF4E00193E6
:1066980001930193019305E00093DA0108951FEF38
:1066A80008950A811B812C813D816091FF04772721
:1066B800060F171F271F371F000F111F221F331F19
:1066C8007A830B831C832D8300E00F9376DF0F9171
:1066D800112339F40A95C9F7112319F406E0009338
:1066E800DA010FEFECEAF4E00193019301930193CF
:1066F800089522E030E0E4E2F4E061917191361708
:106708003707A1F43297122F1A9502E40E944C37EA
:10671800A12F102F0A2F085D1B4F01931193F80129
:1067280022E430E031932A95E9F708952A9529F76C
:1067380010E000E008950881198122E0E4E2F4E025
:10674800619171910617170731F4329710E0119390
:1067580011931FEF08952A9599F710E0089528815D
:106768003981222339F4332329F404E00093DA0130
:1067780010E0089502E0E4E2F4E0619171912617D7
:10678800370711F41FEF08950A95B9F704E000934D
:10679800DA0110E00895E7EFF4E0019111912191F9
:1067A800319108951091DA0100E00093DA0108951B
:1067B800A80111274117510749F00EEA14E00150CA
:1067C80010400000E1F741505040B9F708951123F7
:1067D80031F00EE00A950000E9F71A95D1F708950F
:1067E8001127A081B181A20FB31F30F0A617B707F8
:1067F80009F010F41FEF02C0A62FB72FA083B183B2
:1068080008952150304018F011911D93FACF089542
:1068180047FC7894F999FCCFF894F999F9CF089541
:10682800F7DF4F93E1BDF2BDF89A000040B51417A9
:1068380019F010BDFA9AF99A4F9147FC7894089587
:10684800E7DFE1BDF2BDF89A000010B547FC789487
:106858000895312FFF91EF910F91BF91AF91EF9371
:10686800FF930023D1F0FD01772311F4108102C0BA
:106878000E942434112389F0332379F0101768F02B
:106888002227E00FF21F232F200F422F211B30F069
:1068980029F0021B772311F40C930895131B772317
:1068A80011F41C9300C03327A40FB31F219523951F
:1068B800772301F01D9111932A95E1F708953F91EF
:1068C8002F910F91BF91AF91FF91EF912F933F932C
:1068D800892F8370882359F0869539F41F930E9475
:1068E8002434312F1F91319603C0359101C0319165
:1068F800332331F0892F807101F02C91011708F4AE
:106908000895402F411B542F431B58F1211730F491
:10691800632F620F061708F0062F23C0AF93BF93AB
:10692800EF93FF93522F511B541708F4452F552707
:10693800A10FB51FA40FB51F1196FD01E30FF51F99
:10694800542F5395892F807101F00E9002925A9519
:10695800E1F7FF91EF91BF91AF91012F030F040F62
:1069680011F4340F3395892F807101F00C9322278D
:10697800A10FB21F892F8370882349F0869529F4C7
:106988000E942434012E319603C0059001C0019065
:10699800892F807101F00D923A9561F70895332798
:1069A8002227BB27AA2746FA26F40E9424343196C8
:1069B80001C01191112319F4112700270895512FAF
:1069C800002311F0539571C046FA26F40E9424342E
:1069D800319601C01191E89442F81D3261F45A953C
:1069E80059F3689442F846FA26F40E942434319602
:1069F80001C0119111C01B3261F45A95E9F2E89473
:106A080042F846FA26F40E942434319601C01191C6
:106A180003C0143209F449C0052F0A956AF25527B4
:106A28007727992788270F9308C00F9346FA26F4EB
:106A38000E942434319601C01191103310F11A3399
:106A480000F51053412F8D01000F111F771F991F5B
:106A5800000F111F771F991F0A0F1B1F781F981F00
:106A6800720F931F000F111F771F991F040F151F17
:106A7800781F981FD801272F392F0F910A954AF0B0
:106A8800D4CF0F91689441F8112700273327222784
:106A980008958D0142FA46F40150104020403040DC
:106AA80020953095109500950895E89442F85A95E8
:106AB800D9F3593038F746FA26F40E94243431962F
:106AC80001C01191113608F010521033D8F21A3360
:106AD80028F01134B8F21734A8F6175F1F7004E0D5
:106AE800AA0FBB1F221F331F0A95D1F7A12B5A9556
:106AF80011F7CFCF1127B081BB2389F0662309F4A2
:106B08006395B61760F0E60FF11F6A95B61B162F4E
:106B18001395A1910A1719F0BA95D1F7112708957D
:106B2800112389F0B081BB2371F0B01B60F0B395DD
:106B3800AA27E00FFA1FB11708F0B12F11910E9490
:106B4800F736BA95D9F7089515910E94F736BA9590
:106B5800D9F708951191112331F0B12F11910E94A5
:106B6800F736BA95D9F70895BF91AF91EF914F9144
:106B78005F911F91AF93BF93CF93DF932797E894CB
:106B880042F8AA27A8835D834E83EF9304E60E9408
:106B9800563725D0102F0AE00E94563720D0102FE4
:106BA8001ED05F91FF91EF91EF93FF93DE012E814D
:106BB8003D8199C00D911D910E94F7363A9519F4BF
:106BC8001EE20E94F7360A95B1F7FF91EF9108810E
:106BD8000083098101830A810283EF010895E88116
:106BE800EE2311F4112339F0E395E883FF27EC0F26
:106BF800FD1F106310830895BF91AF91EF914F91DE
:106C08005F913F912F911F910F91AF93BF93CF93B6
:106C1800DF932E97AA27A8835C874D87EF93EEE032
:106C2800F2E7A801B901E89442F845FA16F437FDED
:106C380042F819E01F93A591B59115910591EF932D
:106C4800FF93E12FF02F0E940D38B001AC01102FF7
:106C580011230AF41195C3DFFF91EF911F911A9543
:106C680049F7182FBCDF5F91FF91EF91EF93FF93E6
:106C7800DE012D853C8537C0BF91AF91EF914F91D3
:106C88005F911F910F91AF93BF93CF93DF93299794
:106C9800AA27A8835F834887EF93E2E2F2E7D80147
:106CA800E89442F845FA16F417FD42F864E0259195
:106CB80035913296EF93FF930E948737DF01102FAB
:106CC80011230AF411958BDFFF91EF916A9579F7FB
:106CD8001A2F85DF5F91FF91EF91EF93FF93DE010C
:106CE80028853F8100C00881002321F4039508838B
:106CF80010E31983239700810883018109830281A6
:106D08000A833323B9F12223A9F14C913A95431709
:106D180040F0342F321B42FA1EF41DE20E94F7366F
:106D280049CF042F241714F0022F039542FA0EF4CA
:106D38003A95152F031B019531F02AF00E94F7367A
:106D48003A950A95D9F742FA1EF41DE20E94F736E1
:106D5800321B241770F010E30E94F7361EE20E94DF
:106D6800F7363327241B29F010E30E94F7362A95BB
:106D7800D9F720CF42FA16F43A954AF00C91301B15
:106D880031F028F0152F0E94F7363A95E1F742FACC
:106D98001EF41DE20E94F7360DCF0D9144FC02C08F
:106DA800019001C00590001511F0989408950023F2
:106DB80011F4189408950A951D9144FC02C001909D
:106DC80001C00590101599F398940895B2E0429582
:106DD800142F1F701A3008F0195F105D0E94F736E3
:106DE800BA95A9F70895EF93FF9343FADEF01F933E
:106DF800E981FA811881112331F41F91689441F8CF
:106E0800FF91EF9108951A9518831F9146FA16F08D
:106E1800119303C00E9414343196FA83E983FF91D9
:106E2800EF910895E881F9811F930F932F933F9372
:106E3800AF93BF936F937F934F935F938F939F937A
:106E480009959F918F915F914F917F916F91BF911C
:106E5800AF913F912F910F911F91FF91EF9108955D
:106E6800212F102F222339F0283010F011270895F0
:106E7800110F2A95E9F70895212F102F222339F0B1
:106E8800283010F01127089516952A95E9F70895E6
:106E9800109F102D012D08953F912F91012F1F91C3
:106EA8002F933F93332729E0111F2A9511F4032FBD
:106EB8000895331F301B18F4300F8894F5CF0894C9
:106EC800F3CF9801442745FA86F4BD013702F00153
:106ED800269F80013603F40B100DE11DF41F720389
:106EE800F40B100DE11DF41F08953B9FF0012A9F3C
:106EF80080013A9F100DE11DF41F2B9F100DE11D1D
:106F0800F41F08959801552745FA96F45B2F432FEF
:106F18004B27E89447FF45F837FF04C0219509F44B
:106F28003A953095B7FF04C0A19509F4BA95B09584
:106F3800EE27FF1B11E1AA1FBB1F1A9541F48D0113
:106F480045FA26F4019509F41A9510950895EE1F4F
:106F5800FF1FE21BF30B20F4E20FF31F8894EBCF23
:106F68000894E9CFD801F9011F910F917F916F9192
:106F78005F914F910F931F9302C0D801F90145FA11
:106F8800CEF48F2F8727E89487FF45F8F7FF08C0CE
:106F9800A095B095E095F095AF5FBF4FEF4FFF4FCD
:106FA80077FF08C040955095609570954F5F5F4F8B
:106FB8006F4F7F4F992788271124002410E2769578
:106FC80067955795479520F48A0F9B1F0E1E1F1E25
:106FD800179407949795879577956795579547954B
:106FE8001A9589F78A019B0145FA46F40150104029
:106FF8002040304020953095109500950895D8018F
:10700800F9011F910F917F916F915F914F910F93AC
:107018001F93112745FAD6F4172F8F2F8727E89447
:1070280087FF45F8F7FF08C0A095B095E095F09563
:10703800AF5FBF4FEF4FFF4F77FF08C040955095A8
:10704800609570954F5F5F4F6F4F7F4F1F938827F5
:1070580099270024112411E2441F551F661F771F2A
:107068001A9571F48A019B0145FA46F401501040C3
:107078002040304020953095109500955F910895F7
:10708800881F991F001C111C8A1B9B0B0E0A1F0AC4
:1070980030F48A0F9B1F0E1E1F1E8894DDCF0894A4
:1070A800DBCF222349F0203118F01127002708955B
:1070B800169507952A95E1F70895EE2369F0E032D1
:1070C80028F011270027222733270895369527957A
:1070D80017950795EA95D1F70895222349F02031AD
:1070E80018F0112700270895000F111F2A95E1F7BE
:1070F8000895EE2369F0E03228F0112700272227AF
:1071080033270895000F111F221F331FEA95D1F767
:1071180008951770E6E0F2E70024E10FF01DC89526
:107128001C9110291C9308951F70183010F01196A7
:107138001850E6E0F2E70024E10FF01DC89511278A
:107148000C91202F002101131FEF08951770E6E01E
:10715800F2E70024E10FF01DC8951127082D002142
:1071680009F0109508951770E6E0F2E70024E10FA2
:10717800F01DC895302D30951127092D002109F0F3
:107188001095F894092D0323902E47FC78940895C0
:1071980011271093090008951C91011711F4112764
:1071A8000895F89413951D93ED91FC917193F5173B
:1071B80021F4E41711F4FD013396FC93EE931FEFCD
:1071C80047FC789408951C911123E9F3F8947723E8
:1071D80011F41A951C931396ED91FC911191772354
:1071E80051F4B801F51721F4E41711F4FD013196B3
:1071F800FC93EE938B0147FC78940895189501024F
:1072080004081020408000CA9A3B00E1F5058096EA
:10721800980040420F00A086010010270000E803F4
:107228000000640000000A00000000015C01200268
:107238003A20042E6D703306504C41593A200841CB
:107248004354494F4E3A20073A20726561647910D9
:107258004552524F523A206E6F7420666F756E64B5
:107268000F414354494F4E3A2053746F7070656410
:10727800032A2E2A054449523A200646494C453AE3
:10728800200C564F4C554D453A20564F4C3D08530F
:1072980054415455533A202453595354454D3A2098
:1072A800436F6E6669726D20466C61736820446F27
:1072B800776E6C6F6164204D6F6465200E5359536F
:1072C80054454D3A204163746976651053595354B7
:1072D800454D3A2061626F727465642E16455252AC
:1072E8004F523A20556E6B6E6F776E20436F6D6DFF
:1072F800616E6414494E49543A204D50336F72619F
:10730800746F722056312E320C494E49543A20443B
:1073180053502048570C494E49543A204453502062
:1073280053570C494E49543A205344636172640BD5
:10733800494E49543A205265616479052A2E6D7088
:10734800331B494E49543A2052656164792C206EAA
:107358006F2066696C657320666F756E642245528E
:10736800524F523A2049444520696E69742066613B
:10737800696C65642C206E6565642052657365745C
:107388000E414354494F4E3A20506175736564135A
:107398004552524F523A20436172642072656D6FB4
:1073A8007665640C000D000E000F000B0009000646
:1073B80000030000000800050002000A000700049E
:1073C8000001001B001C001D001E001A00180015FB
:1073D8000012000000170014001100190016001315
:1073E80000100007496E69744453500000000749B3
:1073F8006E697449444500000007496E6974464146
:10740800540000000449646C650000000000000995
:107418005374617274506C61790007506C617969BA
:107428006E67000000095061757365506C617900E2
:1074380006506175736564000000000753746F702F
:10744800706564000000054572726F7200000000EC
:1074580000025041000000001002504600000000E9
:107468001102504E000000001202534600000000B6
:107478001902534E000000001A0253500000000089
:1074880015025053000000001302434F0000000093
:107498001402444900000000200246490000000090
:1074A8002102565500000000160256440000000054
:1074B8001702565300000000180242500000000056
:1074C800800249440000000081025354000000007B
:1074D800A002464100000000A1025544000000003F
:0174E800A201
:027DFE0055AA84
:100000000C94CB2F0C9402390C9402390C940239C5
:100010000C9402390C9402390C9402390C94023974
:100020000C9402390C9402390C9402390C94023964
:100030000C9402390C9402390C9402390C94023954
:100040000C9402390C9402390C946A300C940239E5
:100050000C9440310C940E310C9402390C940239FA
:100060000C9402390C9402390C9402390C94023924
:0C0070000C9402390C9402390C940239F3
:00000001FF
